:100000000C9473000C949B000C949B000C949B002C
:100010000C949B000C9483090C949B000C949B0003
:100020000C949B000C949B000C949B000C949B00E4
:100030000C949B000C949B000C949B000C949B00D4
:100040000C94C61E0C949B000C94081C0C94E21B90
:100050000C949B000C949B000C949B000C949B00B4
:100060000C94C01C0C949B0089128B128D128F1261
:100070009112931295129712C812CB12CE12C5127A
:10008000D112D412E612E61200000000240027006C
:100090002A0000000000250028002B0000000000BE
:1000A00023002600290004040404040404040202BA
:1000B00002020202030303030303010204081020E7
:1000C00040800102040810200102040810200000F2
:1000D0000008000201000003040700000000000007
:1000E00000005E2F483011241FBECFEFD8E0DEBFE6
:1000F000CDBF26E0AEE7B4E001C01D92A73EB20737
:10010000E1F714E0A0E0B1E0EEE0FFE602C0059008
:100110000D92AE37B107D9F710E0C2E7D0E004C0C6
:100120002197FE010E94D333C137D107C9F70E943E
:10013000101F0C947A370C9400000F931F930E94A9
:100140001419009193041091940420919504309116
:100150009604DC01CB01801B910BA20BB30B853FF6
:100160009140A105B10508F4DEC161E080E00E9484
:10017000450B82EC93E00E94700E60919B0670919B
:100180009C0680919D0690919E0642E00E9401137C
:1001900083E394E00E94700E809188048130C1F462
:1001A0000E94A41E60E080E00E94450B8EEC93E06C
:1001B0000E94700E8091910490919204909301019D
:1001C0008093000160E071E084E690E00E945B1E95
:1001D000809188048230D1F50E94A41E60E080E006
:1001E0000E94450B80EE93E00E94700E8091910476
:1001F00090919204909348018093470120910001CF
:1002000030910101821B930B63E070E00E947E330A
:10021000260F371F3093440120934301260F371FC9
:10022000309346012093450163E471E087E690E056
:100230000E945B1E65E471E08AE690E00E945B1E0E
:1002400067E471E08DE690E00E945B1E8091880477
:100250008330D1F50E94A41E60E080E00E94450B2F
:1002600081EF93E00E94700E80919104909192042E
:1002700090934E0180934D012091470130914801A8
:10028000821B930B63E070E00E947E33260F371FC2
:1002900030934A0120934901260F371F30934C01B8
:1002A00020934B0169E471E080E790E00E945B1EBF
:1002B0006BE471E083E790E00E945B1E6DE471E007
:1002C00086E790E00E945B1E809188048430D1F51F
:1002D0000E94A41E60E080E00E94450B82E094E052
:1002E0000E94700E80919104909192049093540119
:1002F0008093530120914D0130914E01821B930B4D
:1003000063E070E00E947E33260F371F3093500168
:1003100020934F01260F371F309352012093510134
:100320006FE471E089E790E00E945B1E61E571E097
:100330008CE790E00E945B1E63E571E08FE790E040
:100340000E945B1E80918804853009F048C00E949D
:10035000A41E60E080E00E94450B83E194E00E94CF
:10036000700E809191049091920490935C0180931F
:100370005B012091530130915401821B930B97FD37
:1003800003969595879595958795280F391F3093F6
:10039000560120935501280F391F3093580120939F
:1003A0005701820F931F90935A018093590165E57D
:1003B00071E082E890E00E945B1E67E571E085E8ED
:1003C00090E00E945B1E69E571E088E890E00E9481
:1003D0005B1E6BE571E08BE890E00E945B1E8091F4
:1003E0008804863009F048C00E94A41E60E080E0C6
:1003F0000E94450B84E294E00E94700E809191046B
:1004000090919204909364018093630120915B0129
:1004100030915C01821B930B97FD03969595879510
:1004200095958795280F391F30935E0120935D01C4
:10043000280F391F3093600120935F01820F931FB3
:1004400090936201809361016DE571E08EE890E028
:100450000E945B1E6FE571E081E990E00E945B1EE7
:1004600061E671E084E990E00E945B1E63E671E062
:1004700087E990E00E945B1E80918804873009F034
:1004800048C00E94A41E60E080E00E94450B85E306
:1004900094E00E94700E8091910490919204909348
:1004A0006C0180936B012091630130916401821B88
:1004B000930B97FD03969595879595958795280FAE
:1004C000391F3093660120936501280F391F30933F
:1004D000680120936701820F931F90936A018093B4
:1004E000690165E671E08AE990E00E945B1E67E6BB
:1004F00071E08DE990E00E945B1E69E671E080EAA0
:1005000090E00E945B1E6BE671E083EA90E00E943F
:100510005B1E0E941419609393047093940480935B
:100520009504909396041F910F9108958F929F9236
:10053000AF92BF92FF920F931F93CF93DF93EC0183
:10054000F090A2040091A8041091A904F110A0C099
:100550000230110509F49CC08130910509F04BC0AF
:10056000809188048F5F873008F087E0809388044B
:1005700040913F01509140016091410170914201D1
:100580008091820190918301A0918401B0918501B5
:10059000840F951FA61FB71F80938201909383013C
:1005A000A0938401B09385016091820170918301D1
:1005B000809184019091850120913F01309140010B
:1005C000409141015091420180903F019090400143
:1005D000A0904101B09042010E949233C501B40144
:1005E0000E946E3360938201709383018093840133
:1005F000909385014DC0019609F04AC040913F019A
:1006000050914001609141017091420180918201BD
:1006100090918301A0918401B0918501841B950B79
:10062000A60BB70B8093820190938301A093840162
:10063000B093850160918201709183018091840162
:100640009091850120913F013091400140914101FD
:100650005091420180903F0190904001A090410153
:10066000B09042010E949233C501B4010E946E33E2
:10067000609382017093830180938401909385013C
:10068000809188048150823008F481E0809388044E
:100690008091820190918301A0918401B0918501A4
:1006A00081309846A948B94060F080E098E6A9E812
:1006B000B9E08093820190938301A0938401B09369
:1006C00085018091820190918301A0918401B09174
:1006D0008501803A9648A140B10560F480EA96E829
:1006E000A1E0B0E08093820190938301A093840104
:1006F000B093850121E0F21249C0C130D10509F55E
:1007000080913F0190914001A0914101B09142013F
:1007100040918D0450918E0460918F0470919004EB
:10072000840F951FA61FB71F80938D0490938E048E
:10073000A0938F04B09390040130110509F07EC09E
:10074000B0C2CF3F8FEFD80709F540913F015091DC
:100750004001609141017091420180918D0490911E
:100760008E04A0918F04B0919004841B950BA60B6E
:10077000B70B80938D0490938E04A0938F04B09355
:1007800090040130110509F059C09CC201301105D7
:1007900009F054C08091A4049091A504A091A604EE
:1007A000B091A7048093820190938301A093840168
:1007B000B0938501C130D105C1F46DE671E08AE1E5
:1007C00090E00E94021E40913F01509140016091D3
:1007D000410170914201FC0180819181A281B3812C
:1007E000840F951FA61FB71F1BC0CF3FFFEFDF076A
:1007F00029F56DE671E08AE190E00E94021E4091C9
:100800003F01509140016091410170914201FC0112
:1008100080819181A281B381841B950BA60BB70BBC
:1008200080936D0190936E01A0936F01B09370015E
:100830006DE671E08AE190E00E94281E8091A80494
:100840009091A904029709F073C0C130D10541F518
:100850008091A4049091A504A091A604B091A7044E
:100860008093820190938301A0938401B0938501CA
:1008700068E974E085E190E00E94021E40913F012A
:10088000509140016091410170914201FC018081D1
:100890009181A281B381840F951FA61FB71F31C01C
:1008A000CF3FFFEFDF0709F043C08091A404909190
:1008B000A504A091A604B091A7048093820190930F
:1008C0008301A0938401B093850168E974E085E118
:1008D00090E00E94021E40913F01509140016091C2
:1008E000410170914201FC0180819181A281B3811B
:1008F000841B950BA60BB70B181619061A061B06B8
:100900004CF480937D0190937E01A0937F01B0937E
:10091000800108C010927D0110927E0110927F012B
:10092000109280016DE771E085E190E00E94281E41
:100930008091A8049091A904039709F040C0809188
:10094000A4049091A504A091A604B091A70480935B
:10095000820190938301A0938401B0938501C130FB
:10096000D10591F48093820190938301A093840137
:10097000B093850161E573E08DEF95E00E948C1BDB
:1009800081E08093810115C0CF3FFFEFDF0709F0C1
:100990005DC08093820190938301A0938401B09302
:1009A00085016DE473E08DEF95E00E948C1B109241
:1009B000810161E871E08DE090E00E94821E8091EB
:1009C000A8049091A904049709F040C08091A40460
:1009D0009091A504A091A604B091A70480938201F0
:1009E00090938301A0938401B0938501C130D10518
:1009F00091F48093820190938301A0938401B0933A
:100A0000850161E573E083E096E00E948C1B81E044
:100A10008093A00415C0CF3F2FEFD20709F090C0FC
:100A20008093820190938301A0938401B093850108
:100A30006DE473E083E096E00E948C1B1092A004AA
:100A400060EA74E080E090E00E94821E8091A80439
:100A50009091A904059709F073C0C130D10541F503
:100A60008091A4049091A504A091A604B091A7043C
:100A70008093820190938301A0938401B0938501B8
:100A800065E771E088E290E00E94021E40913F011C
:100A9000509140016091410170914201FC018081BF
:100AA0009181A281B381840F951FA61FB71F31C00A
:100AB000CF3FFFEFDF0709F043C08091A40490917E
:100AC000A504A091A604B091A704809382019093FD
:100AD0008301A0938401B093850165E771E088E20A
:100AE00090E00E94021E40913F01509140016091B0
:100AF000410170914201FC0180819181A281B38109
:100B0000841B950BA60BB70B181619061A061B06A5
:100B10004CF48093750190937601A0937701B09384
:100B2000780108C010927501109276011092770139
:100B30001092780165E771E088E290E00E94281E3B
:100B40008091A8049091A904069709F064C0C1306F
:100B5000D10541F58091A4049091A504A091A6042B
:100B6000B091A7048093820190938301A0938401A4
:100B7000B09385016CE974E084E290E00E94021E6B
:100B800040913F01509140016091410170914201BB
:100B9000FC0180819181A281B381840F951FA61FE2
:100BA000B71F2BC0CF3FFFEFDF07A9F58091A4044B
:100BB0009091A504A091A604B091A704809382010E
:100BC00090938301A0938401B09385016CE974E054
:100BD00084E290E00E94021E40913F01509140014A
:100BE0006091410170914201FC0180819181A2815B
:100BF000B381841B950BA60BB70B80939C04909339
:100C00009D04A0939E04B0939F046CE974E084E279
:100C100090E00E94281E8091A8049091A904079753
:100C200079F5CF3FFFEFDF0799F48091A40490910D
:100C3000A504A091A604B091A7048093820190938B
:100C40008301A0938401B09385016DE473E014C027
:100C50002197B1F48091A4049091A504A091A604D9
:100C6000B091A7048093820190938301A0938401A3
:100C7000B093850161E573E087EF95E00E948C1BDE
:100C80008091A8049091A904089769F5DF91CF910C
:100C90001F910F91FF90BF90AF909F908F900C94F9
:100CA0009D008091A4049091A504A091A604B09108
:100CB000A7048093820190938301A0938401B09351
:100CC00085017BCD8091A4049091A504A091A604F8
:100CD000B091A7048093820190938301A093840133
:100CE000B093850186CDDF91CF911F910F91FF9039
:100CF000BF90AF909F908F90089580918B049091BA
:100D00008C04009729F440E95AE36CE170E007C0D5
:100D100081309105A9F440ED51EB67E370E0409319
:100D20008201509383016093840170938501109236
:100D30008D0410928E0410928F041092900448C07B
:100D400082309105A9F440E153E96BE670E04093ED
:100D50008201509383016093840170938501109206
:100D60008D0410928E0410928F041092900438C05B
:100D700083309105A9F440E45BE66AE970E04093B2
:100D800082015093830160938401709385011092D6
:100D90008D0410928E0410928F041092900428C03B
:100DA00084309105A9F440E759EE67ED70E0409377
:100DB00082015093830160938401709385011092A6
:100DC0008D0410928E0410928F041092900420C013
:100DD0008530910529F480E49DE7A4E1B1E01EC0CF
:100DE0008630910529F480ED9FE3A4E4B1E016C0BC
:100DF0008730910529F480E99BE3AEE7B1E00EC0AE
:100E00008830910529F480E290EEA2EBB1E006C0B3
:100E10000997A1F480EC92E3AAE0B3E08093820109
:100E200090938301A0938401B093850110928D0467
:100E300010928E0410928F04109290040895809165
:100E400086049091870461E0019709F446C080E030
:100E50000E94450B80913F0190914001A09141017A
:100E6000B091420184369105A105B10569F188F47C
:100E70008A309105A105B10509F182339105A105DB
:100E8000B105F9F00197A105B10571F586E494E08B
:100E900029C0803127E29207A105B105C1F0803A4F
:100EA00026E8920721E0A207B105A1F0883E934011
:100EB000A105B105C9F48AE594E014C08BE494E07F
:100EC00011C080E594E00EC085E594E00BC08FE58D
:100ED00094E008C084E694E005C080E00E94450BE1
:100EE00089E694E00C94700E0895809189049091A5
:100EF0008A04009739F421E030E03093870420938E
:100F0000860444C08130910589F441E050E060E0FE
:100F100070E040933F015093400160934101709312
:100F20004201109287041092860430C082309105ED
:100F300089F44AE050E060E070E040933F01509354
:100F40004001609341017093420110928704109216
:100F5000860424C08330910589F442E350E060E0C8
:100F600070E040933F0150934001609341017093C2
:100F70004201109287041092860418C084309105B3
:100F800029F484E690E0A0E0B0E016C08530910539
:100F900029F488EE93E0A0E0B0E00EC08630910521
:100FA00029F480E197E2A0E0B0E006C0079781F461
:100FB00080EA96E8A1E0B0E080933F019093400181
:100FC000A0934101B09342011092870410928604CD
:100FD00069E874E087E390E00C945B1ECF92DF92A7
:100FE000EF92FF9261E084E00E94450B60917D01E9
:100FF00070917E0180917F019091800120E432E424
:101000004FE050E00E94B43369017A012093DA0482
:101010003093DB044093DC045093DD042A30310527
:10102000410551051CF480E20E94570BC701B6012F
:101030000E94720E8EE20E94570B60917D017091AA
:101040007E0180917F019091800120E432E44FE0A5
:1010500050E00E94B43328EE33E040E050E00E94BC
:10106000B43369017A012093DA043093DB044093AE
:10107000DC045093DD04243631054105510564F448
:1010800080E30E94570B8AE0C816D104E104F10402
:101090001CF480E30E94570BC701B6010E94720E38
:1010A0008EE20E94570B60917D0170917E018091CC
:1010B0007F019091800128EE33E040E050E00E94F3
:1010C000B4336B017C016093DA047093DB0480938A
:1010D000DC049093DD0484E6C816D104E104F10435
:1010E00064F480E30E94570B8AE0C816D104E1043F
:1010F000F1041CF480E30E94570BC701B6010E9463
:10110000720E8DE494E0FF90EF90DF90CF900C94FE
:10111000700ECF938091A104811114C06EE674E02B
:101120008DE296E00E948C1B1092970410923E0173
:101130006EE371E088E090E00E94821E60E080E152
:101140000E945818C091A104C130A1F46BE973E06A
:101150008DE296E00E948C1BC093970410923E0192
:101160006EE371E088E090E00E94821E60E080E122
:101170000E9458188091A1048230A9F469EB73E0B1
:101180008DE296E00E948C1B81E080933E011092DC
:1011900097046EE371E088E090E00E94821E61E0B7
:1011A00080E10E9458188091A104833080F0109251
:1011B000A1046EE674E08DE296E00E948C1B109212
:1011C0003E016EE371E088E090E00E94821E61EAD9
:1011D00074E085E390E00E94821ECF910C941D0B79
:1011E000CF92DF92EF92FF92CF93DF9360E083E0A4
:1011F0000E94450B80E20E94570B60918201709122
:101200008301809184019091850120E432E44FE0D4
:1012100050E00E94923369017A012A30310518F4B6
:1012200080E20E94570B4AE0C701B6010E94720B90
:101230008EE20E94570B6091820170918301809130
:1012400084019091850120E432E44FE050E00E9457
:10125000923328EE33E040E050E00E94923369017F
:101260007A01E9012436310540F480E30E94570BEE
:101270002A9718F480E30E94570B4AE0C701B60191
:101280000E94720B8EE20E94570B60918201709156
:101290008301809184019091850128EE33E040E044
:1012A00050E00E9492336B017C01EB0164367105C2
:1012B00040F480E30E94570B2A9718F480E30E94C1
:1012C000570B4AE0C701B6010E94720B80E20E94F0
:1012D000570B60E08FE00E94450B63E376E08AE7FE
:1012E00096E00E94D41B60E080E00E94450B6DE216
:1012F00076E08AE796E0DF91CF91FF90EF90DF9064
:10130000CF900C94D41B1F920F920FB60F92112402
:10131000CF92DF92EF92FF920F931F932F933F9301
:101320004F935F936F937F938F939F93AF93BF93ED
:10133000CF93DF93EF93FF9380913B060E942F188A
:10134000EC0180913A060E942F18E0913906EF7067
:10135000CC0FDD1F8C2B94E0E99FF0011124E457A2
:10136000FE4FE80FF11DC081C0933906C07359F1DB
:101370000E94141900917E0410917F042091800432
:10138000309181046B017C01C01AD10AE20AF30A90
:10139000C0928204D0928304E0928404F092850487
:1013A00060937E0470937F04809380049093810403
:1013B000C03119F481E090E004C0C03221F48FEF15
:1013C0009FEF0E949602FF91EF91DF91CF91BF9125
:1013D000AF919F918F917F916F915F914F913F91CD
:1013E0002F911F910F91FF90EF90DF90CF900F9072
:1013F0000FBE0F901F901895FF920F931F93CF93DE
:10140000DF93EC01F62E08811981C8010E94EF31AB
:10141000F81621F06F2DC8010E94F731CE01DF913F
:10142000CF911F910F91FF900895282F30914D0576
:10143000313208F04AC080912A058111FCCF909189
:10144000920642E040932A05209329052FEF20932E
:1014500028051092270530932605EDE2F5E0A6E079
:10146000B5E020E0321721F041914D932F5FFACF84
:101470001092050520910505990F922B9093050573
:1014800090910405913061F4109204059091050546
:101490009093BB009091BC0093FDF8CF95EC01C0F8
:1014A00095EE9093BC0090912A059230E1F39091D3
:1014B00028059F3F79F080912805803241F0809186
:1014C0002805803331F084E005C081E003C082E06C
:1014D00001C083E010922C0510924D0510922B054F
:1014E000089540E0682F8AE796E00C94671CCF933C
:1014F000DF93823028F09091890698609093890656
:1015000080938D0610928E0680E480938F0680E192
:101510008093900680E58093910661E080917E063D
:101520000E94871880917F068F3F19F061E00E942A
:10153000871861E0809180060E948718CAE7D6E08C
:101540009E012A5736408091890684FD03C084E0BD
:1015500090E002C088E090E02196281739072CF42B
:1015600061E08E810E948718EBCF8BE39DE00197AD
:10157000F1F760E080917E060E94581860E080914B
:1015800080060E94581880917F068F3F19F060E016
:101590000E9458188091890684FD20C063E08AE784
:1015A00096E00E943A1CCBE4D6E4CE010197F1F715
:1015B00063E08AE796E00E943A1C2197F1F763E026
:1015C0008AE796E00E943A1C83E592E00197F1F7E2
:1015D00062E08AE796E00E943A1C15C080620E9491
:1015E000710A8BE496E40197F1F780918906806295
:1015F0000E94710A83E592E00197F1F780918906D4
:1016000080620E94710A8091890680620E94710A3C
:1016100084E080938A068CE00E94710A81E00E9437
:10162000710A8BE39FE10197F1F782E080938B06CB
:1016300086E0DF91CF910C94710AEF92FF920F93A5
:101640001F93CF93DF9300D0CDB7DEB78DE2E82EA6
:1016500086E0F82E0EE210E0F70161917F011A8317
:101660000983CE0101960E94FC090F5F1F4F0433CE
:10167000110591F78DE296E00F900F90DF91CF91D9
:101680001F910F91FF90EF900895643008F063E090
:1016900090918D06691710F06FEF690FE62FF0E05B
:1016A000E658F94F9489890F80680C94710A41E0DB
:1016B000682F8AE796E00E94671C81E090E0089519
:1016C000009769F0FC0101900020E9F73197AF0124
:1016D000481B590BBC018AE796E00C94211980E065
:1016E00090E008958F929F92AF92BF920F931F93B5
:1016F000CF93DF93CDB7DEB7A1970FB6F894DEBFD7
:101700000FBECDBF19A2423008F44AE08E010F5D32
:101710001F4F842E912CA12CB12CA50194010E9465
:101720009233E62FB901CA0101501109EA3014F4CD
:10173000E05D01C0E95CD801EC93232B242B252B21
:1017400061F7C8010E94600BA1960FB6F894DEBF46
:101750000FBECDBFDF91CF911F910F91BF90AF9082
:101760009F908F900895CF93C62F91E090932B0573
:1017700090E69093920610922C0510924D05682FDA
:101780008BEE95E00E94BA1A6C2F8BEE95E00E94CA
:10179000BA1A81E0CF910C94150ACF93DF9391E0B0
:1017A00090932B0590E69093920610922C05109240
:1017B0004D05682F8BEE95E00E94BA1A81E00E94D9
:1017C000150A80912A058111FCCF81E080932A05BA
:1017D000109229059FEF90932805109227051092EB
:1017E00026058093050580910505806C809305058D
:1017F00080910405813061F4109204058091050503
:101800008093BB008091BC0083FDF8CF85EC01C0C4
:1018100085EE8093BC0080912A058130E1F38091B0
:101820002705811103C0C091270501C0C1E0E6E092
:10183000F5E0A4EEB4E080E08C1721F091919D9347
:101840008F5FFACF1092E304C093E2048091E30427
:10185000C81731F08BEE95E00E94711AD82FF6CFA1
:101860008D2FDF91CF910895CF93C0E1C80F8C2FBA
:101870000E94CD0B682F63608C2FCF910C94B30B1B
:101880001F93CF93DF93EC01162F83E00E94CD0BC3
:101890009E01332761E070E001C0660F2A95EAF7E8
:1018A000113019F46095682301C0682B83E0DF9143
:1018B000CF911F910C94B30B0F931F93CF93DF9392
:1018C0008B0191E090932B0590E6909392061092F5
:1018D0002C0510924D05682F8BEE95E00E94BA1AE8
:1018E000E801085F1F4F69918BEE95E00E94BA1ADC
:1018F000C017D107C1F781E0DF91CF911F910F9100
:101900000C94150A2F923F924F925F926F927F92A2
:101910008F929F92AF92BF92CF92DF92EF92FF92FF
:101920000F931F93CF93DF93CDB7DEB761970FB6B9
:10193000F894DEBF0FBECDBF2D833E834F83588703
:1019400069877A871C011F870E87609176067091E0
:101950007706809178069091790624E630E040E0A1
:1019600050E00E9441342D87388B4B875C87762E60
:10197000672E582E492E8091700690917106A09185
:101980007206B09173066C017D01FF0CCC08DC2C53
:1019900076019C01AD016C2D7C2D8C2D9C2D0FE1D1
:1019A0000E940C35A12C0AECB02EEAE9CE2EFBE306
:1019B000DF2EE12CF12C00E010E00E946E34AD84AB
:1019C000B888CB84DC84E72CF62C052D142D0E94DE
:1019D000D9330FE10E94273549015A01D501C401CD
:1019E000BB0F880B982FDC0189839A83AB83BC8360
:1019F0009401A5016981762F862F962FAD84B88832
:101A0000CB84DC84E72CF62C052D0E9443352983FA
:101A1000832E942E598B688B7B878C879D872D8195
:101A20003E814F81588569857A85C1012F3FA7E5A1
:101A30003A07A7E44A07A8EF5A07ADE06A0771051D
:101A400081059105A9F0A0F0211534404B46544F73
:101A50006441710581059105B9F0B0F01D8294E0F3
:101A60009E83ABE6AF83B4EFB887E4E1E98709C0B2
:101A70001D82E8E5EE83F7E4FF8328EF28878DE0F9
:101A800089871A86212C312CA980B82CC92CD98899
:101A9000E888FB840C851D852D813E814F8158850A
:101AA00069857A85C1010E949F3429013A01FFE0CE
:101AB0004F1651046104710418F4AFE0AA2E08C057
:101AC0002BE54216510461047104D0F0FAE5AF2E03
:101AD000B12CC12CD12CE12CF12C00E010E029819B
:101AE000382D492D598968897B858C859D850E9473
:101AF000D9332D833E834F83588769877A871C01AA
:101B0000A980B82CC92CD988E888FB840C851D8550
:101B10002D813E814F81588569857A85C1010E945A
:101B20009D34AA24AA94BB24BA94EFE0CE2ED12CE3
:101B3000E12CF12C00E010E00E94D933A980B82CF0
:101B4000C92CD988E888FB840C851D850E949F34A8
:101B5000C901DA010097A105B10529F4C12CD12CE6
:101B60007601C39406C0CC24CA94DC2C5FE0E52E39
:101B7000F12CBC01CD0127E0660F771F881F991F4C
:101B80002A95D1F737E0440C551C661C771C3A9512
:101B9000D1F7A2E05A1A61087108A70196010E94C4
:101BA0009233862E372E982E420E531E641E751EBB
:101BB00084E190E00E9475359A838983FC01D0828C
:101BC000C182862D8370828353824482D701C601ED
:101BD0004CE0B695A795979587954A95D1F7807F64
:101BE000C82EC90CC582368287828E859F85892B37
:101BF00019F4BF018AE107C0AE85BF85119729F4AA
:101C000069817A8182E20E945C0C89819A81619665
:101C10000FB6F894DEBF0FBECDBFDF91CF911F91FD
:101C20000F91FF90EF90DF90CF90BF90AF909F907B
:101C30008F907F906F905F904F903F902F900C947B
:101C40000D361092E3041092E20410922C051092CB
:101C50004D0510922A0581E0809329051092040514
:101C600061E082E10E94581861E083E10E94581807
:101C7000E9EBF0E080818E7F808380818D7F80839F
:101C800088E48093B80085E48093BC008FE59AE1F6
:101C90009093E1048093E00480E69AE19093DF045E
:101CA0008093DE0408950F931F93CF93DF938B01EE
:101CB000877028E0829FC001112480640E94710A0D
:101CC000E801085F1F4F69918AE796E00E94BA1CFD
:101CD000C017D107C1F7DF91CF911F910F910895E0
:101CE0000C94600BCF92DF92EF92FF92CF93DF9331
:101CF00097FF19C06B017C018DE20E94570BEC012C
:101D000066277727CB016C197D098E099F094AE068
:101D10000E94720B8C0F9D1FDF91CF91FF90EF906F
:101D2000DF90CF9008954AE0DF91CF91FF90EF9040
:101D3000DF90CF900C94720B2F923F924F925F9254
:101D40006F927F928F929F92AF92BF92CF92DF92CB
:101D5000EF92FF920F931F93CF93DF93CDB7DEB730
:101D600068970FB6F894DEBF0FBECDBF522E3D87E9
:101D7000442E5E873B011C01A982B98ACA8ADB8A8C
:101D8000EC8AFD8A0E8B1F8B988A8F86211500EABC
:101D900030070CEA400709EB500703E060077105C4
:101DA0008105910511F008F046C02F3F10EE310774
:101DB00015EF410715E05107610571058105910592
:101DC00061F058F02F3F354D41415E47634071054A
:101DD0008105910509F0D8F50BC0512CF1EEFD8776
:101DE000B5EF4B2E05E00E87612C712C212C312C88
:101DF000298139894A895B896C897D898E899F8986
:101E0000A0E00E94553509F0A7C0A52CBD84C42CC4
:101E1000DE847301810120E034E04BE654EF64E19D
:101E200070E080E090E00E949F3429873A874B87DA
:101E30005C87912C24C0512C10EA1D87FCEA4F2EA0
:101E400029EB2E87A3E06A2E712C212C312C2981BD
:101E500039894A895B896C897D898E899F89A0E04F
:101E60000E94553509F0F4C09924939414E0E12EB2
:101E7000F12C00E010E0E986FA860B871C87E984E4
:101E8000FA840B851C85A801970160E070E0CB0106
:101E9000A52CBD84C42CDE847301810129833A837F
:101EA0004B835C836D837E838F83988760E070E0D3
:101EB00080E090E00E94D9332983398B4A8B5B8B79
:101EC0006C8B7D8B8E8B9F8BFF24F3949F1409F476
:101ED000C2C010E0812C912C5401839440E050E06A
:101EE000BA0101C011E0CB01BA0107E0660F771F0C
:101EF000881F991F0A95D1F7C984DA84EB84FC8482
:101F000027E0CC0CDD1CEE1CFF1C2A95D1F7A2E0CB
:101F1000DA1AE108F108A50194010E949233C20E79
:101F2000D31EE41EF51EEF85F889C082D182E282BD
:101F3000F382648375838683978380869186A286E5
:101F4000B3861111BBC0298139894A895B896C89A3
:101F50007D898E899F89B8C0188EA52CBD84C42C1C
:101F6000DE8473018101298139894A895B896C8901
:101F70007D898E899F890E949F3429873A874B8764
:101F80005C8789859A85AB85BC850697A105B105D7
:101F900020F4B6E0AB2EB12C0FC0E984FA840B8597
:101FA0001C8529E0E21627E0F20601051105D0F0B4
:101FB000F8E0AF2EA7E0BA2EC12CD12CE12CF12CE9
:101FC00000E010E0298139894A895B896C897D8923
:101FD0008E899F890E949F34522E3D87442E5E87B2
:101FE0003B011C01A52CBD84C42CDE84730181013E
:101FF000298139894A895B896C897D898E899F8984
:102000000E949D34AA24AA94BB24BA94EFE0CE2E59
:10201000D12CE12CF12C00E010E00E94D933A52C4A
:10202000BD84C42CDE84730181010E949F34A32FE0
:10203000F42FE52F422F5A2F6F2F7E2F4115510578
:1020400061057105F9F4812C912C5401839420C011
:1020500081E0888F82CFAF85B8891D921D921D9235
:102060001C921397FD011482158216821782C12CCF
:10207000D12C7601C3941896CD92DD92ED92FC920C
:102080001B9722C088248A94982C8FE0A82EB12C0C
:10209000F88DF13009F026CFEF85F8891082118292
:1020A00012821382148215821682178281E090E0D8
:1020B000A0E0B0E080879187A287B387252D3D857A
:1020C000442D5E85B301C10168960FB6F894DEBF5A
:1020D0000FBECDBFDF91CF911F910F91FF90EF9079
:1020E000DF90CF90BF90AF909F908F907F906F9038
:1020F0005F904F903F902F900895DF92EF92FF9264
:102100000F931F93CF93DF93FC01E080F180028156
:102110001381D481C581B681D7809701A8016D2F25
:102120007C2F8B2F9D2D35534C405109610971092E
:10213000810991092F3F34434C40510561057105D8
:102140008105910509F098F49701A8016D2F7C2F66
:102150008B2F9D2D07E00E940C3520833183428315
:102160005383648375838683978387E0FDC09701DB
:10217000A8016D2F7C2F8B2F9D2D3A564841510978
:1021800061097109810991092F3F3946484151057B
:10219000610571058105910509F098F49701A80181
:1021A0006D2F7C2F8B2F9D2D06E00E940C352083F8
:1021B000318342835383648375838683978386E068
:1021C000D3C09701A8016D2F7C2F8B2F9D2D345DDF
:1021D0004043510961097109810991092F3F334D2C
:1021E00040435105610571058105910509F098F499
:1021F0009701A8016D2F7C2F8B2F9D2D05E00E944C
:102200000C352083318342835383648375838683B3
:10221000978385E0A9C09701A8016D2F7C2F8B2F94
:102220009D2D385A41465109610971098109910969
:102230002F3F374A414651056105710581059105DA
:1022400009F098F49701A8016D2F7C2F8B2F9D2DFD
:1022500004E00E940C3520833183428353836483DE
:1022600075838683978384E07FC09701A8016D2FD3
:102270007C2F8B2F9D2D3055434C510961097109DD
:10228000810991092F3F3F44434C51056105710578
:102290008105910509F098F49701A8016D2F7C2F15
:1022A0008B2F9D2D03E00E940C35208331834283C8
:1022B0005383648375838683978383E055C0970136
:1022C000A8016D2F7C2F8B2F9D2D305A46485140F1
:1022D00061097109810991092F3F3F4946485140E1
:1022E000610571058105910509F098F49701A80130
:1022F0006D2F7C2F8B2F9D2D02E00E940C352083AB
:10230000318342835383648375838683978382E01A
:102310002BC09701A8016D2F7C2F8B2F9D2D305442
:102320004D40534061097109810991092F3F3F4395
:102330004D405340610571058105910509F098F400
:102340009701A8016D2F7C2F8B2F9D2D01E00E94FE
:102350000C35208331834283538364837583868362
:10236000978381E001C080E0DF91CF911F910F91B1
:10237000FF90EF90DF900895833081F028F4813052
:1023800099F08230A1F008958730A9F08830B9F033
:102390008430D1F4809180008F7D03C080918000D3
:1023A0008F7780938000089584B58F7702C084B5BD
:1023B0008F7D84BD08958091B0008F7703C0809198
:1023C000B0008F7D8093B00008953FB7F89480915E
:1023D000970690919806A0919906B0919A0626B515
:1023E000A89B05C02F3F19F00196A11DB11D3FBF4D
:1023F000BA2FA92F982F8827820F911DA11DB11DDB
:10240000BC01CD0142E0660F771F881F991F4A95D6
:10241000D1F708950F931F93CF938B01C0E1C80F9D
:102420008C2F0E94CD0B0115110511F48F7D04C076
:102430000130110509F48062682F8C2FCF911F9114
:102440000F910C94B30B2F923F924F925F926F9229
:102450007F928F929F92AF92BF92CF92DF92EF9234
:10246000FF920F931F93CF93DF93CDB7DEB72E97D5
:102470000FB6F894DEBF0FBECDBF3C01C982DA8231
:10248000EB82FC820D831E832F83388749875A870E
:102490006B877C878BA18D873C2C2D2C5E2C0E8727
:1024A000412E922EC984DA84EB84FC8484E190E08E
:1024B0000E9475358C01FC01D082C182862D880F67
:1024C000880F880F845D0E94CD0B952D93708C7FB3
:1024D000892BF801828323823482D701C6017CE0F4
:1024E000B695A795979587957A95D1F7807F992D81
:1024F0009F70C92EC80EC58246828E85878398E05C
:1025000069167104B8F4F301EC5CFF4FB8010C9448
:10251000D3338AE20DC082E30BC08AE309C082E4B0
:1025200007C08AE405C082E503C08AE501C08BE5E7
:102530000E945C0C60E1F62EF60C8F2D0E94CD0BF4
:10254000E1E0682FAE1202C0606401C06F7B8F2D86
:102550000E94B30BF1E06F16710459F038F092E06D
:102560006916710449F4A0926F0618C0A0926D0616
:102570000FC0A0926E060FC0E8E06E167104B0F4B2
:10258000F301E45CFF4F0C94D33354E4B52E0EC03A
:102590004CE2B42E0BC034E3B32E08C02CE3B22EB1
:1025A00005C09CE4B92E02C084E5B82E8B2D0E9494
:1025B000CD0B8378FD85F1118C6090E1899E4001FF
:1025C0001124682F68298B2D0E94B30BC8012E9609
:1025D0000FB6F894DEBF0FBECDBFDF91CF911F9134
:1025E0000F91FF90EF90DF90CF90BF90AF909F90B2
:1025F0008F907F906F905F904F903F902F900C94B2
:102600000D368F929F92AF92BF92CF92DF92EF9250
:10261000FF920F931F93CF93DF936B017C01142FD5
:102620009B01AC010E946933882319F082E794E092
:1026300027C046015701E894B7F82FEF3FEF4FE767
:102640005FE7C501B4010E94693381110DC02FEF0E
:102650003FEF4FE75FE7C501B4010E94CB3018168A
:102660001CF486E794E00CC02FEF3FEF4FE75FE4E8
:10267000C701B6010E946433181684F48AE794E017
:10268000DF91CF911F910F91FF90EF90DF90CF904E
:10269000BF90AF909F908F900C94600B2FEF3FEF07
:1026A0004FE75FECC701B6010E94CB3087FDE6CF54
:1026B00020E030E0A901C701B6010E94CB3087FFBE
:1026C00009C08DE20E94570BEC01F7FAF094F7F87D
:1026D000F09402C0C0E0D0E000E060E070E080E094
:1026E0009FE3101741F020E030E040E251E40E9407
:1026F000C3320F5FF6CFA70196010E9457326B01DC
:102700007C010E9435334B015C014AE00E94720B50
:10271000C80FD91F1123A9F1C501B4010E94D030FF
:102720009B01AC01C701B6010E9456326B017C01CE
:102730008EE20E94570BC80FD91F20E030E040E224
:1027400051E4C701B6010E9431314B015C010E9486
:1027500035336B01E12CF12C4AE0C701B6010E9430
:10276000720BC80FD91FC701B6010E94D0309B0160
:10277000AC01C501B4010E9456326B017C011150BD
:10278000E1F6CE01DF91CF911F910F91FF90EF9075
:10279000DF90CF90BF90AF909F908F9008952F9231
:1027A0003F924F925F926F927F928F929F92AF92E1
:1027B000BF92CF92DF92EF92FF920F931F93CF932E
:1027C000DF93CDB7DEB7AA970FB6F894DEBF0FBE82
:1027D000CDBF622E298F732E3A8F4B8F5C8F6D8FFA
:1027E0007E8F8F8F98A319A708A793012F3F34439B
:1027F0004C405105610571058105910509F050F4C2
:10280000198E85E38A8F8CE08B8F1C8E1D8E1E8E19
:102810001F8E18A2298D3A8D4B8D5C8D6D8D7E8D0E
:102820008F8D98A12115304A4C4A594B6340710550
:102830008105910569F060F0198E80EA8A8F8CEA33
:102840008B8F89EB8C8F83E08D8F1E8E1F8E18A24D
:10285000CE0149960E947D108AA7798CBA8DAB8DE6
:10286000FC8DED8D6E8C5F8C48A0272D3B2F4A2F61
:102870005F2F6E2F762D852D942D2F3F05ED300780
:1028800001E140070EE7500703E06007710581058D
:10289000910511F008F07FC09E01235F3F4F490171
:1028A000A12CECE3BE2EF3E5CF2EACE4DA2E10E142
:1028B000E12EF12C00E010E0272D3B2F0E949C0E12
:1028C00088A599A58130910509F44CC038F102978B
:1028D00009F065C3898D809365068A8D80936606AD
:1028E0008B8D809367068C8D809368068D8D809389
:1028F00069068E8D80936A068F8D80936B0688A102
:1029000080936C0680E019A2212C3CE3332E43E532
:10291000442E1CE41CA320E12DA34CC3898D80937D
:1029200055068A8D809356068B8D809357068C8D25
:10293000809358068D8D809359068E8D80935A060C
:102940008F8D80935B0688A180935C0680E019A23E
:10295000212C5CE3352E63E5462E9CE49CA3E0E14C
:10296000EDA328C3898D80935D068A8D80935E06D2
:102970008B8D80935F068C8D809360068D8D809308
:1029800061068E8D809362068F8D8093630688A189
:102990008093640604C3CE010D964C01A12CB12C8A
:1029A000C12CD12CE12CF12C00E010E0272D3B2F85
:1029B0004A2F5F2F6E2F762D852D942D0E949C0E11
:1029C000E8A5F9A5E130F10509F458C020F03297E7
:1029D00009F49AC115C3298D3A8D4B8D5C8D6D8D8F
:1029E0007E8D8E01035F1F4F4801A12CB12CC12C9D
:1029F000D12CE12CF12C00E010E08F8D98A10E94E9
:102A00009C0E1901442E5CA36DA3772E582E692EBF
:102A100060E070E080E090E00E940A12209245069B
:102A200030924606409247061CA1109348062DA1FD
:102A30002093490670924A0650924B0660924C06CB
:102A4000898D809355068A8D809356068B8D809351
:102A500057068C8D809358068D8D809359068E8DE8
:102A600080935A068F8D80935B0688A180935C06C5
:102A700081E031E039A31BA21AA29FC21091750612
:102A8000B98DAA8DFB8DEC8D0D8D09A30E8D0AA33A
:102A90000F8D0EA308A10FA3123009F073C02B2FC6
:102AA0003A2F4F2F5E2F69A17AA18EA1902F305817
:102AB0004A41564061097109810991092F37304E09
:102AC00042475849624071058105910569F160F1FD
:102AD000A0906506B0906606C0906706D090680624
:102AE000E0906906F0906A0600916B0610916C0602
:102AF0002B2F3A2F4F2F5E2F69A17AA18EA19FA174
:102B00000E944C3589F010925D0610925E0610927C
:102B10005F06109260061092610610926206109293
:102B20006306109264066CC220904D0630904E06EB
:102B300040904F06209150062CA3309151063DA3A2
:102B4000709052065090530660905406CE010D9638
:102B50004C015101C42CD22EE32EF72C052D162D3D
:102B60002B2F3A2F4F2F5E2F69A17AA18EA19FA103
:102B70000E949C0E61E070E081E090E00E940A12E9
:102B800019A235C020934D0630934E0640934F0650
:102B900050935006609351067093520680935306EB
:102BA000909354068E01035F1F4F4801A12CB12C56
:102BB000C12CD12CE12CF12C00E010E02B2F3A2F6E
:102BC0004F2F5E2F69A17AA18EA19FA10E949C0E1A
:102BD0001901442E5CA36DA3772E582E692E61E057
:102BE00070E081E090E00E940A1211E019A3298DA3
:102BF0003A8D4B8D5C8D6D8D7E8D8F8D98A130586B
:102C00004A41564061097109810991092F37304EB7
:102C100042475849624071058105910509F008F461
:102C200057C081E080937506209165063091660655
:102C300040916706509168066091690670916A0636
:102C400080916B0690916C06A0E00E94553509F4C6
:102C500042C085E696E00E947D108AA7A0904D06AE
:102C6000B0904E06C0904F06D0905006E0905106AE
:102C7000F09052060091530610915406209165067B
:102C8000309166064091670650916806609169062A
:102C900070916A06CE0101964C0180916B0690916D
:102CA0006C060E949C0E1F928AA4A12CC980DA8017
:102CB000EB80FC800D811E812F81388549855A85E6
:102CC0006B857C8582E090E00E9423120F9003C008
:102CD00088E080937506898D80935D068A8D809348
:102CE0005E068B8D80935F068C8D809360068D8D44
:102CF000809361068E8D809362068F8D809363062C
:102D000088A18093640645C170907506B98DAA8D1F
:102D1000FB8DEC8D0D8D09A31E8D1AA30F8D0EA3B7
:102D200018A11FA301E0701273C02B2F3A2F4F2F51
:102D30005E2F69A17AA18EA1912F30584A41564049
:102D400061097109810991092F37304E424758496D
:102D5000624071058105910569F160F1A0906506F9
:102D6000B0906606C0906706D0906806E09069064D
:102D7000F0906A0600916B0610916C062B2F3A2F8B
:102D80004F2F5E2F69A17AA18EA19FA10E944C3581
:102D900089F01092650610926606109267061092EE
:102DA00068061092690610926A0610926B061092DD
:102DB0006C062AC120904D0630904E0640904F067A
:102DC000209150062CA3309151063DA370905206DD
:102DD0005090530660905406CE010D964C0151015F
:102DE000C42CD22EE32EF72C052D162D2B2F3A2F87
:102DF0004F2F5E2F69A17AA18EA19FA10E949C0EE8
:102E000061E070E082E090E00E940A1219A235C0F1
:102E100020934D0630934E0640934F065093500634
:102E20006093510670935206809353069093540614
:102E30008E01035F1F4F4801A12CB12CC12CD12C56
:102E4000E12CF12C00E010E02B2F3A2F4F2F5E2FBA
:102E500069A17AA18EA19FA10E949C0E1901442E06
:102E60005CA36DA3772E582E692E61E070E082E09E
:102E700090E00E940A1211E019A3298D3A8D4B8D22
:102E80005C8D6D8D7E8D8F8D98A130584A41564056
:102E900061097109810991092F37304E424758491C
:102EA000624071058105910509F008F457C082E080
:102EB0008093750620915D0630915E0640915F0615
:102EC0005091600660916106709162068091630680
:102ED00090916406A0E00E94553509F442C08DE54A
:102EE00096E00E947D108AA7A0904D06B0904E06F5
:102EF000C0904F06D0905006E0905106F0905206D8
:102F0000009153061091540620915D0630915E06A3
:102F100040915F0650916006609161067091620673
:102F2000CE0101964C0180916306909164060E9447
:102F30009C0E1F928AA4A12CC980DA80EB80FC80B1
:102F40000D811E812F81388549855A856B857C8549
:102F500081E090E00E9423120F9003C088E08093EC
:102F60007506898D809365068A8D809366068B8DA4
:102F7000809367068C8D809368068D8D809369069B
:102F80008E8D80936A068F8D80936B0688A18093C7
:102F90006C0681E0E1E0F0E0FBA3EAA30EC080E074
:102FA00019A2212C9CE3392E23E5422EFCE4FCA33C
:102FB00000E10DA3712C512C612C8F938AA4A82EB3
:102FC000CD84DE84EF84F88809891A892B893C89AD
:102FD0004D895E896F89788D88A599A50E942312F5
:102FE0000F9019A1113079F40AA11BA19101442D70
:102FF0005CA16DA1772D852D962D0E94820C03C0BA
:103000007724739401C0712C872DAA960FB6F8947B
:10301000DEBF0FBECDBFDF91CF911F910F91FF900B
:10302000EF90DF90CF90BF90AF909F908F907F9068
:103030006F905F904F903F902F900895009769F0A8
:10304000FC0101900020E9F73197AF01481B590BB3
:10305000BC0185E196E00C942B1B80E00895CF9392
:10306000DF93282F30E0F901E253FF4F8491F901FB
:10307000E654FF4FD491F901EA55FF4FC491CC2398
:1030800091F081110E94BC11EC2FF0E0EE0FFF1FB8
:10309000E456FF4FA591B491EC91ED2381E090E0CF
:1030A00021F480E002C080E090E0DF91CF910895AC
:1030B0001F93CF93DF93282F30E0F901E253FF4FA6
:1030C0008491F901E654FF4FD491F901EA55FF4F7D
:1030D000C491CC23C1F0162F81110E94BC11EC2F9A
:1030E000F0E0EE0FFF1FEE56FF4FA591B4919FB792
:1030F000F894111104C08C91D095D82302C0EC91A2
:10310000DE2BDC939FBFDF91CF911F910895CF936A
:10311000DF9390E0FC01E654FF4F2491FC01EA5557
:10312000FF4F8491882361F190E0880F991FFC0183
:10313000E857FF4FC591D491FC01EE56FF4FA59182
:10314000B491611109C09FB7F894888120958223BA
:103150008883EC912E230BC0623061F49FB7F89402
:103160008881322F309583238883EC912E2B2C93EA
:103170009FBF06C08FB7F894E8812E2B28838FBF9E
:10318000DF91CF9108958E3008F08E508770806463
:1031900080937C0080917A00806480937A00809193
:1031A0007A0086FDFCCF809178002091790090E034
:1031B000922B08958F929F92AF92BF92CF92DF92FF
:1031C000EF92FF926B017C010E94E5114B015C01C3
:1031D000C114D104E104F104F1F00E94E511DC0115
:1031E000CB0188199909AA09BB09883E9340A1051A
:1031F000B10570F321E0C21AD108E108F10888EEA8
:10320000880E83E0981EA11CB11CC114D104E104F6
:10321000F10419F7DDCFFF90EF90DF90CF90BF90D2
:10322000AF909F908F9008952FB7F8946091930678
:103230007091940680919506909196062FBF0895FF
:103240000895CF92DF92EF92FF920F931F93CF9347
:10325000DF936C017A018B01C0E0D0E0CE15DF0571
:1032600081F0D8016D918D01D601ED91FC91019015
:10327000F081E02DC6010995892B11F02196EECF42
:103280007E01C701DF91CF911F910F91FF90EF90C9
:10329000DF90CF900895FC01538D448D252F30E0B1
:1032A000842F90E0821B930B541710F0CF96089553
:1032B00001970895FC01918D828D981761F0828DA0
:1032C000DF01A80FB11D5D968C91928D9F5F9F735A
:1032D000928F90E008958FEF9FEF0895FC01918DFC
:1032E000828D981731F0828DE80FF11D858D90E069
:1032F00008958FEF9FEF0895FC01918D228D892F06
:1033000090E0805C9F4F821B91098F7399270895ED
:103310008EE495E00E947C1921E0892B09F420E0DD
:10332000822F0895FC01848DDF01A80FB11DA35ADF
:10333000BF4F2C91848D90E001968F739927848FD5
:10334000A689B7892C93A089B1898C9183708064F8
:103350008C93938D848D981306C00288F389E02D99
:1033600080818F7D80830895EF92FF920F931F934A
:10337000CF93DF93EC0181E0888F9B8D8C8D981328
:1033800005C0E889F989808185FD26C0F62E0B8D60
:1033900010E00F5F1F4F0F731127E02E8C8DE81286
:1033A0000CC00FB607FCFACFE889F989808185FF48
:1033B000F5CFCE010E949219F1CF8B8DFE01E80F5F
:1033C000F11DE35AFF4FF0829FB7F8940B8FEA8903
:1033D000FB89808180620AC09FB7F894EE89FF89DB
:1033E0006083E889F98980818370806480839FBFCE
:1033F00081E090E0DF91CF911F910F91FF90EF90CE
:103400000895CF93DF93EC01888D8823C9F0EA8972
:10341000FB89808185FD05C0A889B9898C9186FDCD
:103420000FC00FB607FCF5CF808185FFF2CFA889CA
:10343000B9898C9185FFEDCFCE010E949219E7CF1B
:10344000DF91CF91089580E090E0892B29F00E94D0
:10345000881981110C940000089585ED8093BC00BB
:103460008091BC0084FDFCCF10922A050895409104
:10347000BF06262F30E0240F311D21323105DCF448
:1034800020912A052430C9F4FC0180E090E08617E1
:1034900058F43091BF062191DC01A156B94FA30F1A
:1034A000B11D2C930196F3CF8091BF06680F6093F6
:1034B000BF0680E0089581E0089582E008950895B0
:1034C00008950895E091E3048091E204E81730F450
:1034D000F0E0EC51FB4F808190E008958FEF9FEF7B
:1034E00008959091E3048091E204981750F4E92F35
:1034F000F0E0EC51FB4F208130E09F5F9093E304BC
:1035000002C02FEF3FEFC90108958091E20490E0DF
:103510002091E304821B91090895CF92DF92EF92EC
:10352000FF920F931F93CF93DF937C01CB018A010E
:1035300020912B05222389F0EB016B01C40ED51ECF
:10354000CC15DD0569F06991D701ED91FC910190F1
:10355000F081E02DC7010995F3CF642F0E94371A3F
:10356000C801DF91CF911F910F91FF90EF90DF90F5
:10357000CF900895CF93DF931F92CDB7DEB76983C5
:1035800020912B052223D1F020914D05203240F0CF
:1035900021E030E0FC013383228380E090E015C01D
:1035A00080912C05E82FF0E0E35DFA4F998190833C
:1035B0008F5F80932C0580934D0505C061E0CE019F
:1035C00001960E94371A81E090E00F90DF91CF9131
:1035D000089580E090E008950E945C370F931F9358
:1035E000CF93DF93EC0188819981009729F02A819C
:1035F0003B812617370788F48B016F5F7F4F0E944E
:103600009636009761F0998388831B830A832C8107
:103610003D81232B11F4FC01108281E001C080E088
:10362000DF91CF911F910F910895CF93DF93EC011C
:1036300060E08E810E94581861E08E810E945818C7
:1036400060E08E810E9458188BE891E00197F1F7B5
:10365000DF91CF910895EF92FF920F931F93CF9335
:10366000DF936115710511F480E01CC0411551050F
:10367000C1F07B01EC018C819D818A01080F191F2B
:10368000B801CE010E94EE1A882371F32881398196
:103690008C819D81B701820F931F0E9473371D8318
:1036A0000C8381E0DF91CF911F910F91FF90EF90FC
:1036B0000895CF93DF93EC0188819981009711F0F1
:1036C0000E940D36198218821D821C821B821A826A
:1036D000DF91CF910895EF92FF920F931F93CF93B5
:1036E000DF93EC017B018A01BA010E94EE1A81117D
:1036F00004C0CE010E94591B07C01D830C83B70173
:10370000888199810E947337CE01DF91CF911F91FB
:103710000F91FF90EF900895CF93DF93EC01611527
:10372000710559F0FB0101900020E9F73197AF01D5
:10373000461B570B0E946B1B02C00E94591BCE01F7
:10374000DF91CF910895CF93DF93EC01FB018617B2
:10375000970761F0608171816115710529F04481DD
:1037600055810E946B1B02C00E94591BCE01DF9144
:10377000CF910895FC01808191810C940D36FC015C
:1037800011821082138212821582148261157105D2
:1037900051F0FB0101900020E9F73197AF01461B82
:1037A000570B0C946B1B0895DB0114964D915C91A3
:1037B00015976D917C91DC01ED91FC910280F38174
:1037C000E02D09941F920F920FB60F9211242F93A0
:1037D0003F934F935F936F937F938F939F93AF9399
:1037E000BF93EF93FF938EE495E00E949219FF91AF
:1037F000EF91BF91AF919F918F917F916F915F9169
:103800004F913F912F910F900FBE0F901F901895E1
:103810001F920F920FB60F9211242F938F939F93A5
:10382000EF93FF93E0915E05F0915F058081E09159
:103830006405F091650582FD12C090818091670555
:103840008F5F8F7320916805821751F0E0916705B3
:10385000F0E0E25BFA4F958F8093670501C08081AD
:10386000FF91EF919F918F912F910F900FBE0F902D
:103870001F901895CF92DF92EF92FF920F931F93B4
:10388000CF93DF936C017C0187E0E80EF11CC0E070
:10389000D0E0062F10E0B8010C2E02C07595679598
:1038A0000A94E2F76170F70181917F010E94581834
:1038B0002196C430D10579F7C601DF91CF911F91D0
:1038C0000F91FF90EF90DF90CF900C94151BCF924B
:1038D000DF92EF92FF920F931F93CF93DF93EC0150
:1038E000F62E642F8C810E9458188D818F3F19F01D
:1038F00060E00E9458188F850F2D10E084FF25C0CE
:103900006E0187E0C80ED11CE12CF12CB8010E2C01
:1039100002C0759567950A94E2F76170F60181918E
:103920006F010E945818FFEFEF1AFF0A88E0E816AF
:10393000F10461F7CE01DF91CF911F910F91FF90BC
:10394000EF90DF90CF900C94151BB80184E0759533
:1039500067958A95E1F7CE010E943A1C6F2DCE0142
:10396000DF91CF911F910F91FF90EF90DF90CF905B
:103970000C943A1C41E00E94671C81E090E008959D
:103980001F920F920FB60F9211242F933F934F93D4
:103990005F936F937F938F939F93AF93BF93EF93B7
:1039A000FF938091B900887F803609F49CC068F548
:1039B000883209F45BC090F4803109F454C038F4C3
:1039C000882309F4F6C0883009F44DC0F6C0883168
:1039D00009F44CC0803209F45DC0EFC0803409F4B2
:1039E00068C048F4803309F455C0883309F0E5C055
:1039F00080932805D8C0803509F44FC0883509F474
:103A00005DC0883409F0D9C0D6C0883909F4C7C070
:103A1000A8F4883709F467C038F4883609F463C01D
:103A2000803709F460C0C9C0883809F4B8C080394B
:103A300009F45FC0803809F0C0C05BC0803B09F466
:103A400086C038F4803A09F466C0883A09F47FC029
:103A5000B4C0803C09F4A7C0883C09F4A4C0883BEA
:103A600009F48AC0AAC08091050510C0909127056D
:103A700080912605981770F5E091270581E08E0F5B
:103A800080932705F0E0EA5FFA4F80818093BB00C6
:103A900085EC86C0809328058EC0E091270581E0E3
:103AA0008E0F809327058091BB00F0E0EA5FFA4F0C
:103AB000808390912705809126056EC0E0912705AF
:103AC00081E08E0F809327058091BB00F0E0EA5FD4
:103AD000FA4F80838091290581116DC081E0809328
:103AE000040584EA61C083E080932A051092E10610
:103AF000CFCF8091E106803208F051C0E091E1061D
:103B000081E08E0F8093E1068091BB00F0E0EF53DF
:103B1000F94F8083BDCF85EC8093BC0010922A05BD
:103B20008091E106803230F4E091E106F0E0EF535D
:103B3000F94F10826091E10670E0E091DE04F091AF
:103B4000DF0481EC96E009951092E10636C084E02E
:103B500080932A051092C0061092BF06E091E004FF
:103B6000F091E10409958091BF06811105C081E0C3
:103B70008093BF0610929F06E091C00681E08E0FF1
:103B80008093C006F0E0E156F94F80818093BB003E
:103B90009091C0068091BF06981708F479CF85E808
:103BA0008093BC000AC085EC8093BC0010922A056B
:103BB00004C0109228050E942D1AFF91EF91BF9129
:103BC000AF919F918F917F916F915F914F913F91B5
:103BD0002F910F900FBE0F901F9018950F931F936A
:103BE000CF93DF938C01EB010E94EF318883C801F2
:103BF00001960E94EF318983CE01DF91CF911F9111
:103C00000F910895CF92DF92EF92FF920F931F933F
:103C1000CF93DF93EB017B0124E0E20EF11C8B01DB
:103C20006C01C61AD70AC601800F911F0E94EF319E
:103C3000F80181938F01EE15FF05A9F7CE01DF9101
:103C4000CF911F910F91FF90EF90DF90CF9008954B
:103C5000AF92BF92CF92DF92EF92FF920F931F939A
:103C6000CF93DF9300D0CDB7DEB78B016B0124E09B
:103C7000C20ED11C7B015C01A61AB70AC5018E0DCC
:103C80009F1DF70161917F019A838983CE0101967F
:103C90000E94FC09EC14FD0489F7C8010F900F90F5
:103CA000DF91CF911F910F91FF90EF90DF90CF9018
:103CB000BF90AF900895EF92FF920F931F93CF9311
:103CC000DF9300D0CDB7DEB78C017B01FB016081B3
:103CD0009A838983CE0101960E94FC09F7016181D4
:103CE0000F5F1F4F1A830983CE0101960E94FC09C2
:103CF000C7010F900F90DF91CF911F910F91FF900F
:103D0000EF9008950F931F93CF93DF9300D0CDB71B
:103D1000DEB78B01FB0160819A838983CE01019616
:103D20000E94FC09C8010F900F90DF91CF911F9165
:103D30000F910895CF93DF93EB010E94EF318883B9
:103D4000CE01DF91CF9108958FE00E94C318909328
:103D5000920480939104BC01990F880B990B0E94E7
:103D6000D23020E030E040EA50E40E94313120E0DF
:103D700030E040E85AE30E94313160939B06709333
:103D80009C0680939D0690939E0608951F920F9225
:103D90000FB60F9211242F933F938F939F93AF935E
:103DA000BF938091930690919406A0919506B0914F
:103DB00096063091E20623E0230F2D3720F401967A
:103DC000A11DB11D05C026E8230F0296A11DB11D3E
:103DD0002093E2068093930690939406A093950611
:103DE000B09396068091970690919806A0919906B7
:103DF000B0919A060196A11DB11D809397069093EC
:103E00009806A0939906B0939A06BF91AF919F919F
:103E10008F913F912F910F900FBE0F901F9018958B
:103E2000CF93DF93CDB7DEB7AB970FB6F894DEBF75
:103E30000FBECDBF789484B5826084BD84B58160A7
:103E400084BD85B5826085BD85B5816085BD809165
:103E50006E00816080936E001092810080918100DD
:103E600082608093810080918100816080938100D5
:103E7000809180008160809380008091B100846097
:103E80008093B1008091B00081608093B0008091F8
:103E90007A00846080937A0080917A0082608093B7
:103EA0007A0080917A00816080937A0080917A0014
:103EB000806880937A001092C100E0915E05F091D5
:103EC0005F0582E08083E0915A05F0915B051082E6
:103ED000E0915C05F0915D058FEC808310926605A2
:103EE000E0916205F091630586E08083E0916005D2
:103EF000F0916105808180618083E0916005F0919F
:103F00006105808188608083E0916005F0916105A2
:103F1000808180688083E0916005F09161058081F7
:103F20008F7D808382E00E94770A81E00E94710A7F
:103F30008BE39FE10197F1F70E94210E61E08AE097
:103F40000E94871861E08BE00E94871861E08CE096
:103F50000E94871861E08DE00E94871860E08FE082
:103F60000E94871861E080E10E94871861E081E18A
:103F70000E94871862E371E081E00E94530E6AE2BA
:103F800071E082E00E94530E62E271E083E00E94E1
:103F9000530E6AE171E084E00E94530E62E171E029
:103FA00085E00E94530E6AE071E086E00E94530EA5
:103FB00062E071E087E00E94530E6AEA74E089E0F3
:103FC00090E00E949A1EDC018C91813F09F0BAC3F7
:103FD0008EE00E94C318853F91403CF08EE00E9425
:103FE000C3188A3892400CF4ADC360EA74E080E0F4
:103FF00090E00E949A1EDC018C918093A00461E8FD
:1040000071E08DE090E00E949A1EFC018081809317
:10401000810168E974E085E190E00E94021EFC01E4
:1040200080819181A281B38180937D0190937E01F3
:10403000A0937F01B09380016DE671E08AE190E08A
:104040000E94021EFC0180819181A281B381809334
:104050006D0190936E01A0936F01B09370016AE3BC
:1040600071E08FE190E00E94021EFC01808191814D
:10407000A281B3818093820190938301A0938401F4
:10408000B09385016CE974E084E290E00E94021E26
:10409000FC0180819181A281B38180937901909309
:1040A0007A01A0937B01B0937C0165E771E088E21F
:1040B00090E00E94021EFC0180819181A281B38167
:1040C0008093750190937601A0937701B093780166
:1040D0009DE2A92E96E0B92E0EE210E0C8010E94E2
:1040E000EF31D5018D935D010F5F1F4F0433110533
:1040F000A9F76DE276E0CB010E94A31B61EA74E0B0
:1041000085E390E00E949A1EFC0180818093A104C7
:1041100069E874E087E390E00E94EE1DDC018D9178
:104120009C9190938A048093890480916D01909171
:104130006E01A0916F01B091700180937006909311
:104140007106A0937206B09373060E94210E62E975
:1041500087EB0E94B30B8FE00E94CD0B40EC5CEF2D
:104160006BE971E04093760650937706609378068A
:1041700070937906682F6F738FE00E94B30B60E82D
:1041800080E10E94B30B60E881E10E94B30B60E81C
:1041900082E10E94B30B6CE080E10E94B30B6CE003
:1041A00081E10E94B30B6CE082E10E94B30B60E2FC
:1041B00081EB0E94B30B60E881EB0E94B30B00E03F
:1041C00010E020E03CE343E55CE460E170E080E087
:1041D00090E00E94820C61E081E090E00E94400C3F
:1041E00080E090E00E94340C81E090E00E94340C6A
:1041F00082E090E00E94340C68ED71E083E396E089
:104200000E948C1B62E08EE00E94871880916800FB
:1042100084608093680080916D008C6080936D0055
:1042200078940E94141960937E0470937F048093A5
:1042300080049093810488EE93E0A0E0B0E0809346
:10424000820490938304A0938404B09385040E9415
:10425000F00888EEC82E83E0D82EE12CF12C332410
:1042600033946EE371E088E090E00E949A1EFC01B6
:10427000808180933E016AE371E08FE190E00E94CB
:10428000021EFC0180819181A281B38180933A0159
:1042900090933B01A0933C01B0933D01409182017A
:1042A00050918301609184017091850180913A0160
:1042B00090913B01A0913C01B0913D0148175907F5
:1042C0006A077B0731F062E871E08FE190E00E94BD
:1042D000281E8091860490918704019709F093C06D
:1042E0008091820490918304A0918404B09185040C
:1042F00085369105A105B105C0F02AE030E040E027
:1043000050E020933F01309340014093410150938E
:1043100042018EE690E0A0E0B0E0809382049093AA
:104320008304A0938404B0938504809182049091C7
:104330008304A0918404B09185048997A109B109EF
:10434000CC97A105B105C0F422E330E040E050E095
:1043500020933F013093400140934101509342012B
:1043600086E490E0A0E0B0E0809382049093830420
:10437000A0938404B0938504809182049091830477
:10438000A0918404B09185044F97A109B1090A97BF
:10439000A105B105C0F424E630E040E050E02093F0
:1043A0003F0130934001409341015093420183E229
:1043B00090E0A0E0B0E08093820490938304A09307
:1043C0008404B09385048091820490918304A09129
:1043D0008404B09185044F97A105B105A0F4C09263
:1043E0003F01D0924001E0924101F09242012FE062
:1043F00030E040E050E02093820430938304409307
:104400008404509385048091A8049091A904892B79
:1044100011F40E94F0088EE00E94C3188EE00E9402
:10442000C3185C019093AF048093AE046AE070E01F
:1044300080E090E00E94DA188EE00E94C3188EE0BF
:104440000E94C318092E000CAA0BBB0BA5010B2C54
:10445000000C660B770B2C013D0133E0431A510829
:1044600061087108441555056605770564F00396E3
:10447000A11DB11D84179507A607B70724F0B092B8
:10448000B904A092B804A090B804B090B90445E86B
:10449000A41643E0B4066CF01092AD048091AC0415
:1044A00081112FC160E081E10E9458181092D5045B
:1044B00028C158E4A516B10464F48091AD048111BB
:1044C00008C061E081E10E9458183092D504309212
:1044D000AD04C501895491098D34910530F5809161
:1044E000AD04811122C08091AC0481110AC061E049
:1044F00081E10E9458183092AC043092D504309279
:10450000AD048091AD048111FCC01091AC04113058
:1045100009F0F7C060E081E10E9458181092AC04E5
:104520001092D5041093AD04ECC0C50187599109D0
:104530008034910500F58091AD0481111CC08091FB
:10454000A204811108C03092A2043092AD041092EE
:10455000B7041092B6048091AD0481110CC0809113
:10456000A204813041F41092A2048093AD04109211
:10457000B7041092B604C501885D9109C697A8F4E6
:104580008091AD04811111C080918B0490918C04B5
:1045900001968A309105DCF010928C0410928B0405
:1045A0003092AD040E947D06ACC0C5018F50914091
:1045B000C19790F48091AD0481110EC080918B045D
:1045C00090918C04019797FF02C089E090E090934E
:1045D0008C0480938B04E4CFC501815491408C9767
:1045E00000F58091AD0481111CC08091AB04811154
:1045F00004C03092AB043092AD048091AD048111BF
:1046000008C08091AB04813021F41092AB048093F8
:10461000AD048091A1048F5F8093A1040E9489085A
:1046200070C0C5018E5691408297D0F48091AD0440
:10463000811116C08091CB04811104C03092CB044B
:104640003092AD048091AD0481115BC08091CB04A8
:10465000813009F056C01092CB048093AD0451C054
:10466000C501815991408297A8F48091AD048111D0
:1046700011C08091890490918A0401968830910537
:10468000E4F010928A04109289043092AD040E94E2
:10469000750737C0C5018F5A91408336910590F454
:1046A0008091AD0481110EC08091890490918A049B
:1046B000019797FF02C087E090E090938A0480936F
:1046C0008904E3CF83E1A81A82E0B80A97E7A91624
:1046D000B104B8F48091AD04811113C08091A80495
:1046E0009091A90401969093A9048093A804309214
:1046F0008804099724F01092A9041092A80430921B
:10470000AD048091D5048093C4048091820190917E
:104710008301A0918401B091850180349244AF401F
:10472000B10508F4D7C08091820190918301A091D6
:104730008401B0918501803C964CAD42B10508F4EE
:10474000EDC0C8C060EA74E080E090E00E94821E84
:1047500081EF90E09A838983BE016F5F7F4F89E08C
:1047600090E00E945B1E61E871E08DE090E00E94A5
:10477000821E6DE771E085E190E00E94281E6DE6E3
:1047800071E08AE190E00E94281E62E871E08FE10A
:1047900090E00E94281E69E771E084E290E00E94A8
:1047A000281E65E771E088E290E00E94281E0E94C2
:1047B0001D0B61EA74E085E390E00E94821E69E8C7
:1047C00074E087E390E00E945B1E60E071E084E6A5
:1047D00090E00E945B1E63E471E087E690E00E9437
:1047E0005B1E65E471E08AE690E00E945B1E67E470
:1047F00071E08DE690E00E945B1E69E471E080E765
:1048000090E00E945B1E6BE471E083E790E00E9401
:104810005B1E6DE471E086E790E00E945B1E6FE432
:1048200071E089E790E00E945B1E61E571E08CE732
:1048300090E00E945B1E63E571E08FE790E00E94CC
:104840005B1E65E571E082E890E00E945B1E67E513
:1048500071E085E890E00E945B1E69E571E088E800
:1048600090E00E945B1E6BE571E08BE890E00E9497
:104870005B1E6DE571E08EE890E00E945B1E6FE5C7
:1048800071E081E990E00E945B1E61E671E084E9DD
:1048900090E00E945B1E63E671E087E990E00E9471
:1048A0005B1E65E671E08AE990E00E945B1E67E6A8
:1048B00071E08DE990E00E945B1E69E671E080EA9C
:1048C00090E00E945B1E6BE671E083EA90E00E943C
:1048D0005B1E8BCB8091820190918301A09184011A
:1048E000B0918501803C964CAD42B10510F40C941A
:1048F000262E8091820190918301A0918401B09134
:10490000850180349B44AC44B10510F00C94262EF4
:1049100084E085B981E090E00C94212F15B81092C5
:104920008C0410928B0460E070E0CB010E94DA18D6
:104930008091A8049091A904009781F04091820190
:104940005091830160918401709185014093A4048A
:104950005093A5046093A6047093A7042091D504F6
:10496000213009F0CCC0892B09F0C9C0A090B00457
:10497000B090B10485010F5F1F4F1093B1040093F5
:10498000B00484E10E94C318BC01990F880B990BF5
:104990000E94D2304B015C0185E10E94C318BC012A
:1049A000990F880B990B0E94D2302B013C019B017F
:1049B000AC01C501B4010E94643387FD07C061E00A
:1049C00080E00E94450B8AED91E097C0043111050B
:1049D0000CF495C01092B1041092B004A30192019E
:1049E000C501B4010E94573268A779A78AA79BA77F
:1049F000A5019401C301B2010E9456329B01AC0192
:104A000068A579A58AA59BA50E94C3324B015C01CC
:104A100020E030E0A9010E946433181624F0B7FAB0
:104A2000B094B7F8B09420E030E040EA50E4C3011D
:104A3000B2010E94313120E030EC4FE754E40E9493
:104A4000C3322CE238E540EB5CE30E94C3329B01A9
:104A5000AC010E94313120E030E048E452E40E9491
:104A6000C3322B013C0120E030E040E050E4C501BE
:104A7000B4010E94573268A779A78AA79BA7A5010E
:104A8000940160E070E080E89FE30E94C3329B01E4
:104A9000AC0168A579A58AA59BA50E9457329B0108
:104AA000AC0160E070E080E890E40E94C332A301B2
:104AB00092010E9431312B013C0161E080E00E94B3
:104AC000450B8DEE91E00E94700E42E0C501B401ED
:104AD0000E94011361E088E00E94450B82EF91E0A3
:104AE0000E94700E61E08BE00E94450B40E0C30124
:104AF000B2010E94011386EF91E00E94700E91E0D6
:104B00008091A204813009F090E081E02091D504E9
:104B1000211180E0892309F419C18091A8049091A2
:104B2000A904892B09F012C1809171019091720141
:104B3000A0917301B0917401803A56E8950751E055
:104B4000A507B105A4F48091820190918301A09101
:104B50008401B0918501805A9648A140B109B09571
:104B6000A095909581959F4FAF4FBF4F17C0813053
:104B70009846A948B940D4F0809182019091830170
:104B8000A0918401B091850120E038E649E859E020
:104B9000281B390B4A0B5B0BDA01C90180938D048A
:104BA00090938E04A0938F04B09390048091B804E6
:104BB0009091B90487599109C197D0F48091B604B6
:104BC0009091B704843691059CF401969093B704B4
:104BD0008093B604C29761F410928D0410928E04F3
:104BE00010928F04109290041092B7041092B604A1
:104BF0000E941F078090820190908301A090840101
:104C0000B090850180918D0490918E04A0918F04C5
:104C1000B0919004880E991EAA1EBB1E809271014D
:104C200090927201A0927301B092740161E084E0ED
:104C30000E94450B80E20E94570BC501B40120E49D
:104C400032E44FE050E00E94B43349015A0120930E
:104C5000B2043093B3044093B4045093B5043AE0E3
:104C600083169104A104B1041CF480E20E94570B46
:104C7000C501B4010E94720E8EE20E94570B609132
:104C8000710170917201809173019091740120E41F
:104C900032E44FE050E00E94B433A70196010E9435
:104CA000B43349015A012093B2043093B3044093C2
:104CB000B4045093B50444E684169104A104B104ED
:104CC00064F480E30E94570B5AE085169104A10416
:104CD000B1041CF480E30E94570BC501B4010E948B
:104CE000720E8EE20E94570B6091710170917201F9
:104CF0008091730190917401A70196010E94B433D1
:104D00004B015C016093B2047093B3048093B404CC
:104D10009093B50484E688169104A104B10464F468
:104D200080E30E94570B9AE089169104A104B10414
:104D30001CF480E30E94570BC501B4010E94720E5F
:104D400080E20E94570B80E20E94570B91E0809115
:104D5000D504811190E081E02091A204211180E02E
:104D6000892309F42CC28091A8049091A904892B6D
:104D700009F025C263EA72E085E196E00E948C1B8F
:104D80000E94A41E0E9414190E941419809093047A
:104D900090909404A0909504B0909604DC01CB010F
:104DA00088199909AA09BB0984369105A105B1059D
:104DB00010F40C94272F0E941419DC01CB018819E0
:104DC0009909AA09BB0984369105A105B10578F0B6
:104DD0000E941419DC01CB0188199909AA09BB09A1
:104DE000883C9105A105B10510F40C94312F0E9467
:104DF0001419DC01CB0188199909AA09BB09883C5F
:104E00009105A105B10578F00E941419DC01CB01D0
:104E100088199909AA09BB098C329140A105B105ED
:104E200010F40C943B2F0E941419DC01CB0188195B
:104E30009909AA09BB098C329140A105B10578F006
:104E40000E941419DC01CB0188199909AA09BB0930
:104E500080399140A105B10510F40C94452F0E94B2
:104E60001419DC01CB0188199909AA09BB098039F9
:104E70009140A105B10578F00E941419DC01CB0125
:104E800088199909AA09BB09853F9140A105B10577
:104E900010F40C944F2F0E941419DC01CB018819D7
:104EA0009909AA09BB09853F9140A105B10508F4FC
:104EB00084C12091C2043091C3048091C0049091B8
:104EC000C104820F931F2091BE043091BF04820F52
:104ED000931F2091BC043091BD04820F931F209139
:104EE000BA043091BB04820F931F65E070E00E940A
:104EF0007E335B0170939204609391046BE671E0E2
:104F000083EA90E00E94EE1DDC018D919C918A1550
:104F10009B051CF08BEF91E03AC16BE671E083EAF0
:104F200090E00E94EE1DFC0180819181A816B906D7
:104F30001CF488E092E02BC169E671E080EA90E021
:104F40000E94EE1DDC018D919C91A816B9061CF4FF
:104F500085E192E01CC167E671E08DE990E00E9476
:104F6000EE1DFC0180819181A816B9061CF482E235
:104F700092E00DC165E671E08AE990E00E94EE1DC5
:104F8000DC018D919C91A816B9061CF48FE292E089
:104F9000FEC063E671E087E990E00E94EE1DFC012F
:104FA00080819181A816B9061CF48CE392E0EFC0D1
:104FB00061E671E084E990E00E94EE1DDC018D91D4
:104FC0009C91A816B9061CF489E492E0E0C06FE554
:104FD00071E081E990E00E94EE1DFC0180819181E9
:104FE000A816B9061CF486E592E0D1C06DE571E023
:104FF0008EE890E00E94EE1DDC018D919C91A81638
:10500000B9061CF483E692E0C2C06BE571E08BE860
:1050100090E00E94EE1DFC0180819181A816B906E6
:105020001CF480E792E0B3C069E571E088E890E0A5
:105030000E94EE1DDC018D919C91A816B9061CF40E
:105040008DE792E0A4C067E571E085E890E00E94FA
:10505000EE1DFC0180819181A816B9061CF48AE836
:1050600092E095C065E571E082E890E00E94EE1D57
:10507000DC018D919C91A816B9061CF487E992E099
:1050800086C063E571E08FE790E00E94EE1DFC01B1
:1050900080819181A816B9061CF484EA92E077C059
:1050A00061E571E08CE790E00E94EE1DDC018D91DE
:1050B0009C91A816B9061CF481EB92E068C06FE4DD
:1050C00071E089E790E00E94EE1DFC0180819181F2
:1050D000A816B9061CF48EEB92E059C06DE471E09D
:1050E00086E790E00E94EE1DDC018D919C91A81650
:1050F000B9061CF48BEC92E04AC06BE471E083E7E4
:1051000090E00E94EE1DFC0180819181A816B906F5
:105110001CF488ED92E03BC069E471E080E790E028
:105120000E94EE1DDC018D919C91A816B9061CF41D
:1051300085EE92E02CC067E471E08DE690E00E947D
:10514000EE1DFC0180819181A816B9061CF482EF46
:1051500092E01DC065E471E08AE690E00E94EE1DD9
:10516000DC018D919C91A816B9061CF48FEF92E09A
:105170000EC063E471E087E690E00E94EE1DFC0142
:1051800080819181A816B90624F08CE093E00E94FA
:105190001E1861E084E00E94450B65E176E08AE735
:1051A00096E00E94D41B0E9414196093930470939C
:1051B000940480939504909396040E941F07809115
:1051C000A8049091A904181619060CF03AC1019789
:1051D00001F560E080E00E94450B89E193E00E94C8
:1051E000700E0E941F0761E084E00E94450B81EA77
:1051F00092E00E94700E60916D0170916E0180913D
:105200006F01909170010E94720E80ED92E00E94F9
:10521000700E8091A8049091A904029761F40E94F5
:10522000EE0760E080E00E94450B8BE293E00E9475
:10523000700E0E941F078091A8049091A904039703
:1052400059F50E94EE0760E080E00E94450B8CE378
:1052500093E00E94700E80918101811106C06DE47F
:1052600073E08DEF95E00E948C1B8091810181306D
:1052700031F461E573E08DEF95E00E948C1B61E0F5
:1052800080E00E94450B6DEF75E08AE796E00E9492
:10529000D41B80E20E94570B8091A8049091A9042E
:1052A000049771F560E080E00E94450B85E593E08E
:1052B0000E94700E8091A004811106C06DE473E01D
:1052C00083E096E00E948C1B8091A004813031F431
:1052D00061E573E083E096E00E948C1B61E080E072
:1052E0000E94450B80EA92E00E94700E63E076E037
:1052F0008AE796E00E94D41B87E693E00E94700E36
:105300008091A8049091A904059719F560E080E0C8
:105310000E94450B85E793E00E94700E0E941F07D4
:1053200061E084E00E94450B81EA92E00E94700EE9
:10533000609175017091760180917701909178016B
:105340000E94720E86E893E00E94700E80E20E9436
:10535000570B8091A8049091A904069701F560E08D
:1053600080E00E94450B8EE893E00E94700E0E9440
:105370001F0761E084E00E94450B81EA92E00E94F1
:10538000700E60919C0470919D0480919E04909198
:105390009F040E94720E86E893E00E94700E809136
:1053A000A8049091A9040797F1F460E080E00E94BE
:1053B000450B8FE993E00E94700E81EA92E00E9413
:1053C000700E61E080E00E94450B84EC92E00E9448
:1053D000700E67EF75E08AE796E00E94D41B88EBB9
:1053E00092E00E94700E8091A8049091A904089701
:1053F00041F58091FB059091FC05892B11F10091FD
:10540000F7051091F8056DE473E0C8010E946A3752
:10541000892B21F41092A9041092A80461E573E08D
:10542000C8010E946A37892B11F40E949D00809167
:10543000A8049091A904099724F01092A90410924D
:10544000A8049091D4048091A104981731F00E948F
:1054500089088091A1048093D4040E9475076CE9A7
:1054600074E084E290E00E94021EFC018081918140
:10547000A281B3818093790190937A01A0937B01FB
:10548000B0937C0168E974E085E190E00E94021E1F
:10549000FC0180819181A281B38180937D019093F1
:1054A0007E01A0937F01B093800165E771E088E2FF
:1054B00090E00E94021EFC0180819181A281B38153
:1054C0008093750190937601A0937701B093780152
:1054D0001091D504113081F4809182019091830163
:1054E000A0918401B0918501809371019093720124
:1054F000A0937301B0937401409182015091830194
:1055000060918401709185018091CB0440385F499E
:10551000654D7105B0F0811109C068ED71E083E35C
:1055200096E00E948C1B6FEA73E07AC0813049F4E8
:1055300063EB73E083E396E00E948C1B65EB73E002
:1055400018C0409182015091830160918401709153
:10555000850140385F49654D710508F0F2C0811141
:1055600054C063EB73E083E396E00E948C1B6FEA08
:1055700073E081E296E00E948C1B8091A20481304E
:1055800049F44091710150917201609173017091E1
:1055900074010AC081111CC04091820150918301A5
:1055A000609184017091850180917D0190917E01CF
:1055B000A0917F01B0918001840F951FA61FB71F96
:1055C0008093D0049093D104A093D204B093D304D9
:1055D00080919704813009F0B4C0113009F0B1C056
:1055E0004091D0045091D1046091D2047091D304C1
:1055F0008091790190917A01A0917B01B0917C0119
:10560000840F951FA61FB71F94C0813009F099C061
:1056100068ED71E083E396E00E948C1B65EB73E01C
:1056200081E296E00E948C1B8091A2048130A9F552
:105630008090750190907601A0907701B0907801EC
:1056400040917D0150917E0160917F0170918001B8
:105650008091710190917201A0917301B0917401D8
:10566000880D991DAA1DBB1D840F951FA61FB71F6E
:105670008093D0049093D104A093D204B093D30428
:10568000480D591D6A1D7B1D40937D0150937E017D
:1056900060937F017093800132C0811130C04091CE
:1056A0008201509183016091840170918501809005
:1056B000750190907601A0907701B090780180916B
:1056C0007D0190917E01A0917F01B0918001880DB4
:1056D000991DAA1DBB1D480F591F6A1F7B1F4093B0
:1056E000D0045093D1046093D2047093D304809378
:1056F0007D0190937E01A0937F01B0938001809102
:1057000097048130F1F41130E1F48091D00490914C
:10571000D104A091D204B091D30440917901509169
:105720007A0160917B0170917C01841B950BA60B23
:10573000B70B8093D0049093D104A093D204B0937C
:10574000D3048091710190917201A0917301B09185
:1057500074012091CB0480383FE9930735EDA3070E
:10576000B105A0F021110EC02091A204213009F052
:105770008FC040917D0150917E0160917F017091B9
:10578000800158C0213009F083C002C0211136C009
:105790002091A204213009F07BC040917D015091FD
:1057A0007E0160917F0170918001840F951FA61F7B
:1057B000B71F8093D0049093D104A093D204B093E8
:1057C000D30480919704813009F062C0113009F050
:1057D0005FC04091D0045091D1046091D204709187
:1057E000D3048091790190917A01A0917B01B091CD
:1057F0007C01840F951FA61FB71F42C0213009F0FE
:1058000047C02091A204213009F042C040917D019F
:1058100050917E0160917F0170918001840F951FEE
:10582000A61FB71F409175015091760160917701D5
:1058300070917801840F951FA61FB71F8093D00425
:105840009093D104A093D204B093D3048091970491
:105850008130F1F41130E1F48091D0049091D104C1
:10586000A091D204B091D3044091790150917A0172
:1058700060917B0170917C01841B950BA60BB70B8B
:105880008093D0049093D104A093D204B093D30416
:105890008091310690913206892BE1F069EB73E03B
:1058A00080912D0690912E060E946A37892B91F4E3
:1058B000113081F48091820190918301A091840143
:1058C000B09185018093D0049093D104A093D20429
:1058D000B093D3048091A004813029F461E081E089
:1058E00090E00E94400C8091A004811105C060E00E
:1058F00081E090E00E94400C80918101811105C0FF
:1059000060E082E090E00E94400C80918101813053
:1059100029F461E082E090E00E94400C4091D004C4
:105920005091D1046091D2047091D3048091CC0441
:105930009091CD04A091CE04B091CF04481759079F
:105940006A077B0709F053C0209131063091320677
:1059500080912B0690912C062817390709F047C033
:1059600080912D0690912E06609127067091280651
:10597000009719F061157105A1F46115710549F0E1
:10598000232B99F0DB018C9190E091958195910901
:105990000AC0009751F0232B41F0FC01808190E078
:1059A00002C00E946A37892B11F59091CB04809137
:1059B000CA0498131CC09091A2048091C904981342
:1059C00016C040917D0150917E0160917F017091E0
:1059D00080018091C5049091C604A091C704B09144
:1059E000C804481759076A077B0709F42BC160915F
:1059F000D0047091D1048091D2049091D30424E614
:105A000030E040E050E00E94413400E010E00E94AD
:105A1000CF136091820170918301809184019091F4
:105A2000850124E630E040E050E00E94413401E08E
:105A300010E00E94CF1360917D0170917E018091F2
:105A40007F019091800124E630E040E050E00E9428
:105A5000323402E010E00E94CF138091A2048093C0
:105A6000C9048091D0049091D104A091D204B09146
:105A7000D3048093CC049093CD04A093CE04B09330
:105A8000CF046DE276E087E296E00E94A31B80914E
:105A9000CB048093CA048091C4048093D504809180
:105AA0007D0190917E01A0917F01B0918001809352
:105AB000C5049093C604A093C704B093C804609132
:105AC00082017091830180918401909185011BA2D4
:105AD0001AA21DA21CA21FA21EA22AE0AE014F5FA5
:105AE0005F4F0E947F30BE016F5F7F4FCE01829675
:105AF0000E948C1B8091090690910A060097C9F0BC
:105B00006AA17BA16115710591F040910B0650913E
:105B10000C062EA13FA14217530748F00E9473378D
:105B20008EA19FA190930E0680930D0618C00E942F
:105B30000D368AA19BA190930A06809309068CA139
:105B40009DA190930C0680930B068EA19FA190932C
:105B50000E0680930D061BA21AA21DA21CA21FA254
:105B60001EA2CE0182960E94BA1B80910D069091D2
:105B70000E060B9798F51BA21AA21DA21CA21FA22B
:105B80001EA24AE0BE016F5F7F4F80E090E00E945E
:105B90007430BE016F5F7F4FCE0182960E948C1BD6
:105BA00040910D0650910E066091090670910A060B
:105BB000CE0182960E942B1B811104C0CE018296D9
:105BC0000E94591BBE016E5D7F4F89E096E00E94E6
:105BD000A31BCE0182960E94BA1BC7CF6DEB73E068
:105BE000CE0101960E94BF1B40910D0650910E06FA
:105BF0006091090670910A06CE0101960E942B1B46
:105C0000811104C0CE0101960E94591B41E050E071
:105C100060EC73E0CE0101960E942B1B882309F4EF
:105C200048C1BE016F5F7F4F8EE495E00E94D41B98
:105C3000CE0101960E94BA1B64E170E080E090E022
:105C40000E94DA180E94231A0C943121809182015B
:105C500090918301A0918401B091850180349B448F
:105C6000AC44B10590F08091820190918301A091A4
:105C70008401B091850181159241AA47B10528F4AC
:105C800088E085B982E090E0DCC08091820190914B
:105C90008301A0918401B091850181159241AA47A9
:105CA000B10590F08091820190918301A0918401CF
:105CB000B091850181159B41A74BB10528F48CE07B
:105CC00085B983E090E0BDC080918201909183010D
:105CD000A0918401B091850181159B41A74BB1052D
:105CE00090F08091820190918301A0918401B09104
:105CF000850181159442A44FB10528F480E185B94E
:105D000084E090E09EC08091820190918301A091F7
:105D10008401B091850181159442A44FB10590F0A2
:105D20008091820190918301A0918401B0918501BD
:105D3000803C9A4EA142B14028F484E185B985E0C7
:105D400090E07FC08091820190918301A0918401B5
:105D5000B0918501803C9A4EA142B14090F0809173
:105D6000820190918301A0918401B09185018038D6
:105D7000914BAF44B14028F488E185B986E090E0CA
:105D800060C08091820190918301A0918401B091C3
:105D900085018038914BAF44B14068F08091820119
:105DA00090918301A0918401B0918501803C9C4F2A
:105DB000AB49B140F8F08091820190918301A091AC
:105DC0008401B0918501803C9C4FAB49B140B8F053
:105DD0008091820190918301A0918401B09185010D
:105DE00081159A45A246B24050F480E285B988E018
:105DF00090E027C08CE185B987E090E022C08091D7
:105E0000820190918301A0918401B0918501811557
:105E10009A45A246B24010F40C94932480918201DA
:105E200090918301A0918401B0918501813C9B43B5
:105E3000A744B34010F00C94932484E285B989E020
:105E400090E090938C0480938B040C949324809125
:105E50009104909192049093C3048093C2040C9493
:105E6000DB2680919104909192049093C1048093D9
:105E7000C0040C94F7268091910490919204909321
:105E8000BF048093BE040C941327809191049091D9
:105E900092049093BD048093BC040C942F278091AE
:105EA0009104909192049093BB048093BA040C9453
:105EB0004B27CE0101960E94591BB3CECF93DF939F
:105EC000EEE4F5E01382128288EE93E0A0E0B0E009
:105ED00084839583A683B7832CEA31E031832083C2
:105EE00025EC30E03587248724EC30E0378726879F
:105EF00020EC30E0318B208B21EC30E0338B228B97
:105F000022EC30E0358B248B26EC30E0378B268B6F
:105F1000118E128E138E148EEBEEF5E01382128228
:105F200084839583A683B7838EEB91E091838083EE
:105F3000EAE7F6E01382128280ED91E0918380839C
:105F400089E084838FEF8583C8E0C68387E08783F9
:105F500086E0808785E0818784E0828713861486C7
:105F600015861686178681E00E94770AECE3F6E034
:105F7000C0AFC1AF11AA12AA13AA11861286138646
:105F80001486158616861786108A118A128A138A35
:105F9000148A158A168A178A108E118E128E138E05
:105FA000148E158E168E178E10A211A212A213A295
:105FB00014A215A216A217A210A611A612A613A625
:105FC00014A615A616A617A610AA80EC9CEFABE99E
:105FD000B1E082AF93AFA4AFB5AFC9E3D6E083E041
:105FE000898382E08A8360E083E00E94871860E012
:105FF0008A810E94871861E089810E94581861E0B7
:106000008A810E945818188268ED71E083E396E057
:106010000E94BF1B6EE674E08DE296E00E94BF1BFB
:106020006EE674E087E296E00E94BF1B6FEA73E0C1
:1060300081E296E00E94BF1B63EA72E08BE196E08A
:106040000E94BF1B63EA72E085E196E00E94BF1BDD
:1060500063EA72E08FE096E00E94BF1B63EA72E0A1
:1060600089E096E00E94BF1B6DE473E083E096E058
:106070000E94BF1B61E573E08DEF95E00E94BF1B9E
:106080006DE473E087EF95E0DF91CF910C94BF1B37
:1060900087EF95E00E94BA1B8DEF95E00E94BA1B36
:1060A00083E096E00E94BA1B89E096E00E94BA1B4A
:1060B0008FE096E00E94BA1B85E196E00E94BA1B31
:1060C0008BE196E00E94BA1B81E296E00E94BA1B27
:1060D00087E296E00E94BA1B8DE296E00E94BA1B0E
:1060E00083E396E00C94BA1BBB274A3031F4992322
:1060F00022F4BDE2909581959F4F0C94A230BB276E
:10610000FA01A62F6217710581059105330B30FB4B
:1061100066F0AA27660F771F881F991FAA1FA2176C
:1061200010F0A21B63953850A9F7A05DAA3308F0C0
:10613000A95DA19336F7B111B1931082CA010C94F5
:10614000BB30BB27FB015527AA27880F991FAA1F21
:10615000A41710F0A41B83955051B9F7A05DAA3382
:1061600008F0A95DA193009779F7B111B19311924D
:10617000CB010C94BB30DC01FC01672F71917723BC
:10618000E1F7329704C07C916D9370836291AE17F2
:10619000BF07C8F308950E940D3108F481E0089507
:1061A000E89409C097FB3EF49095809570956195B1
:1061B0007F4F8F4F9F4F9923A9F0F92F96E9BB2767
:1061C0009395F695879577956795B795F111F8CFE3
:1061D000FAF4BB0F11F460FF1BC06F5F7F4F8F4F4E
:1061E0009F4F16C0882311F096E911C0772321F044
:1061F0009EE8872F762F05C0662371F096E8862FDC
:1062000070E060E02AF09A95660F771F881FDAF732
:10621000880F9695879597F90895990F0008550F5F
:10622000AA0BE0E8FEEF16161706E807F907C0F01C
:1062300012161306E407F50798F0621B730B840B24
:10624000950B39F40A2661F0232B242B252B21F4FE
:1062500008950A2609F4A140A6958FEF811D811D9E
:1062600008950E9444310C94B5310E94A73138F052
:106270000E94AE3120F0952311F00C949E310C94C5
:10628000A43111240C94E9310E94C63170F3959F1A
:10629000C1F3950F50E0551F629FF001729FBB271D
:1062A000F00DB11D639FAA27F00DB11DAA1F649FB9
:1062B0006627B00DA11D661F829F2227B00DA11D6C
:1062C000621F739FB00DA11D621F839FA00D611DF2
:1062D000221F749F3327A00D611D231F849F600D13
:1062E000211D822F762F6A2F11249F5750409AF03C
:1062F000F1F088234AF0EE0FFF1FBB1F661F771FC8
:10630000881F91505040A9F79E3F510580F00C9492
:106310009E310C94E9315F3FE4F3983ED4F38695C7
:1063200077956795B795F795E7959F5FC1F7FE2B32
:10633000880F911D9695879597F9089597F99F670E
:1063400080E870E060E008959FEF80EC08950024FD
:106350000A941616170618060906089500240A94CA
:1063600012161306140605060895092E0394000C50
:1063700011F4882352F0BB0F40F4BF2B11F460FFDF
:1063800004C06F5F7F4F8F4F9F4F089557FD905808
:10639000440F551F59F05F3F71F04795880F97FBE9
:1063A000991F61F09F3F79F08795089512161306A3
:1063B0001406551FF2CF4695F1DF08C016161706D2
:1063C0001806991FF1CF8695710561050894089507
:1063D000E894BB2766277727CB0197F90895F999A9
:1063E000FECF92BD81BDF89A992780B50895262FDA
:1063F000F999FECF1FBA92BD81BD20BD0FB6F894AA
:10640000FA9AF99A0FBE019608950E944732A59F05
:10641000900DB49F900DA49F800D911D112408959F
:106420002F923F924F925F926F927F928F929F92A4
:10643000AF92BF92CF92DF92EF92FF920F931F9392
:10644000CF93DF93CDB7DEB7CA1BDB0B0FB6F89443
:10645000DEBF0FBECDBF09942A88398848885F8483
:106460006E847D848C849B84AA84B984C884DF80F4
:10647000EE80FD800C811B81AA81B981CE0FD11DD8
:106480000FB6F894DEBF0FBECDBFED010895A29FF9
:10649000B001B39FC001A39F700D811D1124911DF8
:1064A000B29F700D811D1124911D08955058BB2776
:1064B000AA270E946E320C94B5310E94A73138F0A1
:1064C0000E94AE3120F039F49F3F19F426F40C9469
:1064D000A4310EF4E095E7FB0C949E31E92F0E9465
:1064E000C63158F3BA17620773078407950720F07F
:1064F00079F4A6F50C94E8310EF4E0950B2EBA2F42
:10650000A02D0B01B90190010C01CA01A0011124B9
:10651000FF27591B99F0593F50F4503E68F11A1665
:10652000F040A22F232F342F4427585FF3CF4695F6
:1065300037952795A795F0405395C9F77EF41F1618
:10654000BA0B620B730B840BBAF09150A1F0FF0FE2
:10655000BB1F661F771F881FC2F70EC0BA0F621FCE
:10656000731F841F48F4879577956795B795F795BE
:106570009E3F08F0B0CF9395880F08F09927EE0F53
:106580009795879508950E94D7320C94B5310E9453
:10659000AE3158F00E94A73140F029F45F3F29F056
:1065A0000C949E3151110C94E9310C94A4310E9449
:1065B000C63168F39923B1F3552391F3951B550B1D
:1065C000BB27AA2762177307840738F09F5F5F4FC6
:1065D000220F331F441FAA1FA9F335D00E2E3AF005
:1065E000E0E832D091505040E695001CCAF72BD01D
:1065F000FE2F29D0660F771F881FBB1F261737076E
:106600004807AB07B0E809F0BB0B802DBF01FF279F
:1066100093585F4F3AF09E3F510578F00C949E31AD
:106620000C94E9315F3FE4F3983ED4F38695779577
:106630006795B795F7959F5FC9F7880F911D969558
:10664000879597F90895E1E0660F771F881FBB1FB4
:10665000621773078407BA0720F0621B730B840B61
:10666000BA0BEE1F88F7E09508950E94CE3188F0AE
:106670009F5798F0B92F9927B751B0F0E1F0660F06
:10668000771F881F991F1AF0BA95C9F714C0B13047
:1066900091F00E94E831B1E008950C94E831672F41
:1066A000782F8827B85F39F0B93FCCF38695779576
:1066B0006795B395D9F73EF490958095709561955F
:1066C0007F4F8F4F9F4F08950E940D3108F48FEF39
:1066D00008950E940D31880B990B0895DB018F936B
:1066E0009F930E940532BF91AF91A29F800D911D93
:1066F000A39F900DB29F900D1124089597FB072E34
:1067000016F4009407D077FD09D00E94613507FC8C
:1067100005D03EF4909581959F4F089570956195B1
:106720007F4F0895A1E21A2EAA1BBB1BFD010DC0CD
:10673000AA1FBB1FEE1FFF1FA217B307E407F50731
:1067400020F0A21BB30BE40BF50B661F771F881F0D
:10675000991F1A9469F760957095809590959B01A3
:10676000AC01BD01CF010895052E97FB1EF40094E6
:106770000E94CB3357FD07D00E94923307FC03D011
:106780004EF40C94CB3350954095309521953F4F66
:106790004F4F5F4F089590958095709561957F4F0D
:1067A0008F4F9F4F0895EE0FFF1F0590F491E02D3E
:1067B0000994DF93CF931F930F939A9DF02D219F00
:1067C000F00D8B9DF00D8A9DE02DF10D039FF00DD6
:1067D000029FE00DF11D4E9DE00DF11D5E9DF00D3F
:1067E0004F9DF00D7F936F93BF92AF925F934F9346
:1067F000D5010E9447328B01AC01D7010E9447327C
:10680000EB01E80FF91FD6010E9429342F913F9127
:10681000D6010E944732C60FD71FE81FF91FAF915C
:10682000BF910E9429342F913F910E944732C60F99
:10683000D71FE81FF91FD6010E944732E60FF71F46
:106840009801BE01CF0111240F911F91CF91DF91CB
:1068500008950E944732460F571FC81FD91F08F4DA
:106860003196089597FB57FF0C9442349F938F9372
:106870000E9442346E1B7F0BAF91BF918A0B9B0B22
:106880000895E894DF93CF93FC01DB010E94473227
:106890007F936F93E9019A01AC01BF93AF933F934C
:1068A0002F93DF010E94473226F46C1B7D0B820B75
:1068B000930B9E01EB01FC010E942934AF91BF9123
:1068C0002F913F910E942934BE01CF01F9012F91F0
:1068D0003F91CF91DF910895689401C0E894F92F1A
:1068E000F12B12F00C94A034A0E0B0E0EAE7F4E35E
:1068F0000C941632092E059422F40E94FC341123C4
:1069000092F4F0E80F26FFEFE094F09400951095D4
:10691000B094C094D094A194BF0ACF0ADF0AEF0AC2
:10692000FF0A0F0B1F0B0E94AB3407FC0E94FC34C4
:10693000CDB7DEB7ECE00C943232689401C0E89435
:106940008F929F92CF93DF930E94AB34DF91CF91D0
:106950009F908F90089588249924F401E401B0E475
:106960009F93AA279A158B049C04ED05FE05CF057D
:10697000D007A10798F4AD2FDC2FCF2FFE2FE92DE4
:10698000982C892E982F872F762F652F542F432FE1
:10699000322F2227B85031F7BF9127C01B2EBF914D
:1069A000BB27220F331F441F551F661F771F881FE9
:1069B000991F881C991CEE1FFF1FCC1FDD1FAA1FEB
:1069C000BB1F8A149B04EC05FD05CE05DF05A0075F
:1069D000B10748F08A189B08EC09FD09CE09DF09C8
:1069E000A00BB10B21601A94E1F62EF49401AF01D3
:1069F000BE01CD01000C089560957095809590952D
:106A000030954095509521953F4F4F4F5F4F6F4FB9
:106A10007F4F8F4F9F4F08950F93083090F0982F1E
:106A2000872F762F652F542F432F322F2227085080
:106A3000F4CF220F331F441F551F661F771F881F77
:106A4000991F0A95B2F70F91089597FB10F81694C5
:106A500000080F93083098F00850232F342F452F4B
:106A6000562F672F782F892F902DF4CF0594979567
:106A700087957795679557954795379527950A9503
:106A8000AAF70F9108952A0D3B1D4C1D5D1D6E1D2B
:106A90007F1D801F911F08952A153B054C055D053C
:106AA0006E057F058007910708950024A7FD0094D7
:106AB0002A173005400550056005700580059005D2
:106AC0000895AA1BBB1B51E107C0AA1FBB1FA61735
:106AD000B70710F0A61BB70B881F991F5A95A9F787
:106AE00080959095BC01CD0108950F931F93CF938E
:106AF000DF938230910510F482E090E0E091E506AA
:106B0000F091E60620E030E0A0E0B0E0309719F127
:106B1000408151810281138148175907C8F08417B9
:106B2000950769F4109731F012960C93129713960B
:106B30001C9327C00093E5061093E60622C021159A
:106B4000310519F04217530718F49A01BD01EF01FE
:106B5000DF01F801DBCF21153105F9F0281B390BD6
:106B60002430310580F48A819B816115710521F003
:106B7000FB019383828304C09093E6068093E5062D
:106B8000FE01329644C0FE01E20FF31F8193919300
:106B900022503109398328833AC02091E30630918D
:106BA000E406232B41F42091880130918901309330
:106BB000E4062093E3062091860130918701211598
:106BC000310541F42DB73EB740918A0150918B01B8
:106BD000241B350BE091E306F091E406E217F3077E
:106BE000A0F42E1B3F0B2817390778F0AC014E5F3D
:106BF0005F4F2417350748F04E0F5F1F5093E40690
:106C00004093E3068193919302C0E0E0F0E0CF016E
:106C1000DF91CF911F910F910895CF93DF9300974C
:106C200009F481C0FC01329713821282A091E5061B
:106C3000B091E606109781F420813181820F931F75
:106C40002091E3063091E4062817390751F5F093B7
:106C5000E406E093E30667C0ED0120E030E0CE17E4
:106C6000DF0740F44A815B819E0141155105F1F037
:106C7000EA01F5CFD383C28340815181840F951FF0
:106C8000C817D90759F488819981840F951F0296F6
:106C9000918380838A819B8193838283211531052F
:106CA00029F4F093E606E093E5063DC0E901FB8395
:106CB000EA8349915991C40FD51FEC17FD0761F480
:106CC00080819181840F951F0296E90199838883C1
:106CD000828193819B838A83E0E0F0E012968D911C
:106CE0009C911397009719F0FD01DC01F7CF8D916E
:106CF0009C9111979D012E5F3F4F820F931F209112
:106D0000E3063091E4062817390769F4309729F42F
:106D10001092E6061092E50602C013821282B0932A
:106D2000E406A093E306DF91CF910895A0E0B0E0E0
:106D3000ECE9F6E30C941432EC01009721F4CB015A
:106D40000E947535B4C0FC01E60FF71F9C0122506C
:106D50003109E217F30708F4A8C0D9010D911C917D
:106D6000119706171707B0F00530110508F49BC0FE
:106D7000C80104978617970708F495C002501109B7
:106D8000061B170B019311936D937C93CF010E9407
:106D90000D3689C05B01A01AB10A4C01800E911E0C
:106DA000A091E506B091E606612C712CE12CF12C46
:106DB000109709F446C08D919C911197A815B905BB
:106DC000B1F56C0142E0C40ED11CCA14DB0478F1A9
:106DD0004C018A189B08640142E0C40ED11C129633
:106DE000BC9012971396AC91B5E0CB16D10440F04D
:106DF000B282A38391828082D9016D937C9309C072
:106E00000E5F1F4F800F911FF90191838083EB2D3F
:106E1000FA2FE114F10431F0D7011396FC93EE93AD
:106E2000129741C0F093E606E093E5063CC0681671
:106E3000790608F43C017D0112960D90BC91A02DBD
:106E4000B7CF8091E3069091E40688169906E1F4A5
:106E500066167706C8F480918601909187010097A5
:106E600041F48DB79EB740918A0150918B01841BEC
:106E7000950BE817F907C8F4F093E406E093E306EE
:106E8000F901718360830FC0CB010E9475357C01CD
:106E9000009759F0A801BE010E946137CE010E94FF
:106EA0000D36C70104C0CE0102C080E090E0CDB72E
:106EB000DEB7EEE00C94303281E090E0F8940C9470
:106EC0007A37FB01DC0102C001900D924150504025
:106ED000D8F70895FB01DC018D9101908019011014
:106EE000D9F3990B0895FB01DC0101900D9200206C
:106EF000E1F7089510E0C2E7D0E004C0FE010E946F
:0E6F0000D3332196C337D107C9F7F894FFCFDA
:106F0E00A5031F1115111D1D111F1F11151115158B
:106F1E00111F1F111D1D1D1D1D1F1F1117111515D1
:106F2E00111F1F1117111D1D111F1F1515111D1DCD
:106F3E001D1F1F111D111D1D111F70E9D70001E826
:106F4E00030000940384034E03E40276021C02E065
:106F5E0001C201A701970189017901620158014718
:106F6E00013A013101290112010D010501EC9D02C9
:106F7E000040420F00B80B0000A8FDFFFF183D8730
:106F8E00000170E9D7000000E7068000000204004F
:106F9E0003000110030200000302010006000400BA
:106FAE00060500200605040000000000B419211992
:106FBE004B19011A7C195A196E1900000000BA1AE1
:106FCE008D1AE91A611A851A711A621A00000000E8
:106FDE00BA1C2119E91A20195500535752202020A6
:106FEE00202020503D305720202020200053575283
:106FFE003D0020503D005720202000FFFFFFFFFFE7
:10700E00FFFFFF072B363000FFFFFFFFFFFFFFFFE5
:10701E00072B353500FFFFFFFFFFFFFFFF072B3567
:10702E003000FFFFFFFFFFFFFFFF072B343500FF90
:10703E00FFFFFFFFFFFFFF072B343000FFFFFFFFB7
:10704E00FFFFFFFF072B333500FFFFFFFFFFFFFFA3
:10705E00FF072B333000FFFFFFFFFFFFFFFF072B64
:10706E00323500FFFFFFFFFFFFFFFF072B3230001F
:10707E00FFFFFFFFFFFFFFFF072B313500FFFFFF75
:10708E00FFFFFFFFFF072B313000FFFFFFFFFFFF6A
:10709E00FFFF072B352000FFFFFFFFFFFFFFFF075E
:1070AE0020202000FFFFFFFFFFFFFF0620202020F3
:1070BE0000FFFFFFFFFFFF05202020202000FFFF25
:1070CE00FFFFFF0420202020202000FFFFFFFF03F2
:1070DE002020202020202000FFFFFF022020202043
:1070EE002020202000FFFF01202020202020202013
:1070FE002000FFFF2020202020202020202000FF25
:10710E002020202020202020202020002020202091
:10711E00202020202020202000436F72722E504C01
:10712E004C2053693533353120200020436F727265
:10713E006563742E2042464F2D32200020202020E1
:10714E0020434C4B202D203220202020004F6666FD
:10715E00004F6E2000202020434C4B31203D3E201E
:10716E0056464F2020200020203E20434C4B2D31F0
:10717E002020202000436F72722E46696C74657257
:10718E002073697A6500487A202020202000204351
:10719E006F72722E20536869667420435720004325
:1071AE006F72722E20535F4C4556454C2D3F004C4E
:1071BE005342004C0055534200414D2000464100C1
:1071CE003B00202050494E204130203D20003020F1
:1071DE0042616C6C203D204F46462056464F2000A3
:1071EE00332042616C6C3D20302E38206D6B562062
:1071FE0000362042616C6C3D2036206D6B5620208F
:10720E002000392042616C6C3D203530206D6B566C
:10721E00202000392B323064423D20353030206D35
:10722E006B562000392B343064423D2035303030DF
:10723E00206D6B5600392B363064423D2035303090
:10724E0030306D6B560031487A20003130487A006C
:10725E003530487A003130304800316B487A003191
:10726E00306B48003130306B004175746F005353F2
:0E727E0042006E616E00696E66006F766600FB
:00000001FF
